S01A00005333324B3134365F626F6F746C6F616465722E73726563E2
S113000000F000201104000059040000590400000D
S113001059040000590400005904000000000000C5
S1130020000000000000000000000000590400006F
S1130030590400000000000059040000015D0000A4
S1130040213800002B380000353800003F3800000C
S113005049380000533800005D380000673800005C
S1130060713800007B380000853800008F380000AC
S113007099380000A3380000AD380000B7380000FC
S1130080C13800005904000059040000590400005C
S113009059040000590400005904000059040000E8
S11300A05904000059040000FB4000000541000011
S11300B00F410000590400005904000059040000D5
S11300C059040000590400005904000059040000B8
S11300D059040000590400005904000059040000A8
S11300E05904000059040000590400005904000098
S11300F05904000059040000590400005904000088
S11303F0590400005904000059040000FFFFFFFFE6
S1130400FFFFFFFFFFFFFFFFFFFFFFFFFE7FFFFF79
S113041072B64FF000014FF000024FF000034FF0AE
S113042000044FF000054FF000064FF00007B846F7
S1130430B946BA46BB46BC4604488546044880478C
S11304400448804762B605F0BBFCFEE700F00020DC
S1130450491B0000791B0000FFF7FEBF53B94AB9DE
S1130460002908BF00281CBF4FF0FF314FF0FF30B8
S113047000F07EB9ADF1080C6DE904CE00F006F889
S1130480DDF804E0DDE9022304B070472DE9F0470C
S1130490089D04468E46002B4ED18A4294466DD95F
S11304A0B2FA82F757B1C7F1200EB94020FA0EFE16
S11304B002FA07FC4EEA010E00FA07F44FEA1C495F
S11304C0210CBEFBF9F61FFA8CF809FB16EE41EA83
S11304D00E4106FB08F38B420AD91CEB010106F11D
S11304E0FF3280F027818B4240F22481023E614436
S11304F0C91AA4B2B1FBF9F009FB101144EA014492
S113050000FB08F8A0450AD91CEB040400F1FF33F2
S113051080F00E81A04540F20B810238644440EA29
S11305200640A4EB080400267DB1FC4000232C60A7
S11305306B603146BDE8F0878B4209D9002D00F08D
S11305401481002685E8030030463146BDE8F08773
S1130550B3FA83F6002E40F090808B4202D382429D
S113056000F2FD80841A61EB030101208E46002D08
S1130570EBD085E810403146BDE8F0871AB94FF05A
S1130580010CBCFBF2FCBCFA8CF7A7BBA1EB0C037F
S11305904FEA1C421FFA8CF80126B3FBF2FE210C31
S11305A002FB1E3341EA034108FB0EF38B4208D9D8
S11305B01CEB01010EF1FF3002D28B4200F2D1801C
S11305C08646C91AA3B2B1FBF2F002FB101143EA4A
S11305D0014408FB00F8A04508D91CEB040400F111
S11305E0FF3302D2A04500F2B7801846A4EB0804FA
S11305F040EA0E4098E7C7F1200301FA07F40CFA29
S113060007FC20FA03FED9404FEA1C424EEA040ECE
S1130610B1FBF2F64FEA1E4302FB16111FFA8CF8E7
S113062043EA014306FB08F1994200FA07F40AD9A8
S11306301CEB030306F1FF3080F08C80994240F2FA
S11306408980023E63445B1A1FFA8EF1B3FBF2F019
S113065002FB103341EA034100FB08F38B4208D943
S11306601CEB010100F1FF3E70D28B426ED90238BF
S11306706144CB1A40EA06468FE7C6F1200722FA06
S113068007F8B34001FA06F448EA030320FA07FC2A
S11306904FEA134EF9404CEA040CB1FBFEF94FEA61
S11306A01C440EFB19111FFA83F844EA014109FBAB
S11306B008F48C4202FA06F200FA06FA08D959182C
S11306C009F1FF3044D28C4242D9A9F102091944FC
S11306D0091B1FFA8CFCB1FBFEF00EFB10114CEA57
S11306E0014400FB08F8A04507D91C1900F1FF31AB
S11306F02AD2A04528D902381C4440EA0940A4EB78
S11307000804A0FB02894C45C446494616D313D0BD
S113071055B1BAEB0C0364EB010404FA07F7F34098
S11307201F43F4402F606C6000263146BDE8F0871B
S11307301846F4E61646DBE6C245E9D2B8EB020CED
S113074069EB03010138E3E70846D6E7704690E712
S11307508146BDE7064676E70238644446E73046FC
S113076005E7AEF1020E61442BE72E462846ECE67F
S1130770704700BF000000000000000000000000FF
S113078001F0FF01102A2BDB10F0070F08D010F83E
S1130790013B013A8B422DD010F0070F42B3F6D142
S11307A0F0B441EA012141EA014122F007047FF05B
S11307B000070023F0E80256083C85EA010586EAB2
S11307C0010685FA47F5A3FA87F586FA47F6A5FAEE
S11307D087F68EB9EED1F0BC01F0FF0102F00702FA
S11307E032B110F8013B013A83EA010313B1F8D1A5
S11307F00020704701387047002D06BF3546033886
S1130800073815F0010F07D1013015F4807F02BFBE
S1130810013015F4C03F0130F0BC0138704700BF0F
S1130820022800D9704708B501F060F808BD022815
S113083000D9704710B5044601F088F8204601F04D
S113084011F810BD022801D90020704708B501F045
S11308509FF808BD022800D9704708B501F018F8C0
S113086008BD022800D9704708B500F0FBFF08BD99
S1130870E1B130B4421E4B1E10FA83F40020082567
S113088041F2210101E0A24212D012F8013F80EAB4
S113089003202B4610F4004F14BF81EA40004000AF
S11308A080B2013B9BB2002BF4D1ECE708467047C1
S11308B030BC70472DE9F04F83B004460E4698468D
S11308C00025AA4B1D60AA4B1D60AA4B1D60AA4BB4
S11308D01D60AA4B1D804FF480522946A84805F09C
S11308E08CFA55222946A74805F087FA012E02D032
S11308F0A54EB71CAFE02046FFF7B3FF40F2054218
S11309002946A14805F079FA43212046FFF7A2FFC2
S1130910EEE79D4B9B78002B00F09B82994901F8F0
S1130920023F9A48032310F8012F22B101F8012F46
S113093001339BB2F7E701339BB200218C4A11606B
S1130940832B24D8904AD75C8DF80770A7F1300226
S1130950D2B2092A1BD8002002468B4E012502EB95
S1130960820207EB4202303A01339BB2842B0BD054
S1130970F75C2846A7F13001C9B20929EFD97C4BAD
S11309801A608DF8077002E0794B1A6088B9794BC8
S113099018684044784B1860754B196800F0D2FC15
S11309A0734B1B68B3F5001F40F2A98003B0BDE888
S11309B0F08F8DF80770EAE79DF80730022B29D0F5
S11309C002A901F8015D2046FFF72AFF9DF80730D0
S11309D0012BF1D1842231462046FFF728FF8021E4
S11309E03846FFF745FF96F8822096F8833003EBEC
S11309F002239BB298428CD040F2054229463046ED
S1130A0005F0FBF92046FFF72CFF15212046FFF7E0
S1130A1021FFD1E740F2044231462046FFF707FFA9
S1130A204FF480613846FFF723FF96F8022496F8C6
S1130A30033403EB02239BB298420ED040F20542EA
S1130A400021304605F0D9F92046FFF70AFF1521A9
S1130A502046FFF7FFFE0025B2E74B4B9B78002BA7
S1130A6000F0FC81474800F8023F4849032303E0B3
S1130A7000F8012F01339BB211F8012F002AF7D19E
S1130A8001339BB200213A4A116040F2034293427F
S1130A9024D83D4AD05C8DF80700A0F13002D2B2D0
S1130AA0092A1BD800252A4640F20446DFF8D8C09C
S1130AB0012702EB820200EB4202303A01339BB27F
S1130AC0B34215D01CF803003D46A0F13001C9B271
S1130AD00929EED9264B1A608DF80700254B1868B2
S1130AE04044254B1860224B196800F02BFC57E753
S1130AF01F4B1A60002DF1D08DF80700EEE740F28D
S1130B0005420021204805F078F906212046FFF728
S1130B10A1FE43212046FFF79DFE0027174B1F80AF
S1130B20124E194D05F102092FE18422294620466F
S1130B30FFF77DFE80214846FFF79AFE95F8822054
S1130B4095F8833003EB02239BB2984220D040F205
S1130B5005420021284605F050F92046FFF781FEA2
S1130B6015212046FFF776FE0FE100BF5C10002040
S1130B70580000206810002064100020601000203D
S1130B805C000020000000206C1000206E1000208B
S1130B90D6F800B0B44BD3F800A0D34528BF002347
S1130BA01BD2B24B1B88B24A284610F8021FD154FC
S1130BB099180AF1FF3E9E44AEEB0B0E96447F3328
S1130BC003EB020C01238E4507D010F8012F01F826
S1130BD0012F01339BB28C45F5D1A4490A881A44EC
S1130BE00A809B44C6F800B040F205420021284622
S1130BF005F003F9D34513D09E4B1B689B4504D9DC
S1130C00ABEB030BBBF5805F2ED040F20542002115
S1130C10284605F0F2F806212046FFF71BFEB4E053
S1130C20944B1B68534504D2AAEB0303B3F5805FCE
S1130C3007D906212046FFF70DFE022F40F0A580BC
S1130C40B4E6DFF834A24FF48052DAF80010884892
S1130C5000F09CFB3368874A13604344CAF80030B1
S1130C600022824B1A80E4E7DFF80CA24FF4805292
S1130C70DAF800107E4800F089FB7E4A136803F519
S1130C80805313604344CAF800300022774B1A8023
S1130C90BBE740F2044229462046FFF7C8FD4FF463
S1130CA080614846FFF7E4FD95F8022495F8033483
S1130CB003EB02239BB298420DD040F2054200217F
S1130CC0284605F09AF82046FFF7CBFD152120466B
S1130CD0FFF7C0FD59E0D6F800A0634B1B689A45A6
S1130CE028BF00231BD2614A1188614AAC461CF814
S1130CF0020F5054881803F1FF3E8E44AEEB0A0EE7
S1130D00964401F2FF3111440123864507D01CF8B3
S1130D10012F00F8012F01339BB28142F5D15349D1
S1130D200A881A440A8053443360524A1268934230
S1130D3003D99B1AB3F5805F0DD040F20542002120
S1130D40284605F05AF82046FFF78BFD0621204679
S1130D50FFF780FD19E0DFF820A14FF48052DAF8A4
S1130D600010434800F012FB424A136803F5805315
S1130D7013604344CAF8003000223C4B1A80DCE77D
S1130D803268394B1B689A423ED002A9002301F80D
S1130D90013D2046FFF744FD9DF80730013B172B2A
S1130DA0F3D801A252F823F02B0B0000930C00009F
S1130DB08B0D0000810D00008B0D00008B0D0000D9
S1130DC08B0D00008B0D00008B0D00008B0D0000BF
S1130DD08B0D00008B0D00008B0D00008B0D0000AF
S1130DE08B0D00008B0D00008B0D00008B0D00009F
S1130DF08B0D00008B0D00008B0D00008B0D00008F
S1130E008B0D0000AD090000A7B1012FBDD140F248
S1130E1005420021284604F0F0FF2046FFF721FD9B
S1130E2006212046FFF716FD43212046FFF712FD59
S1130E300227AAE740F205420021284604F0DDFF1C
S1130E402046FFF70EFD15212046FFF703FD01277D
S1130E509BE70022044B1A60032373E50022024B34
S1130E601A60032315E600BF58000020601000201C
S1130E705C000020681000206410002008B50A49B6
S1130E80062001F09BFE0949002001F097FE084965
S1130E90012001F093FE0749022001F08FFE04F0C7
S1130EA02BFC054B187008BDE44E0020DC4E0020DE
S1130EB0D84E0020E04E0020084F00204368B3F1D4
S1130EC0FF3F0DD080B500AF02684FF000504FF0E7
S1130ED0E021C1F8080D82F3088872B6984780BDF6
S1130EE0704700002DE9F84F43210020FFF7B2FCC2
S1130EF043210120FFF7AEFC00229A4B1A601A46E8
S1130F001368B3F5C87FFBD90020FFF79BFC842846
S1130F1066D90022944B1A600122944B1A60322045
S1130F2002F004FF924B1B68002211468E480068B1
S1130F30FFF7C0FC00228B4B1A60322002F0EAFE5D
S1130F40884A1368632BFCD9322002F0EFFE864CEA
S1130F508849206800F0A8FC8749206800F0A4FCB8
S1130F60864B1A688649206800F09EFC854B1A68F7
S1130F708549206800F098FC844B1A6884492068ED
S1130F8000F092FC834B1A688349206800F08CFCC3
S1130F90824B1A788249206800F086FC2468012C70
S1130FA014BF002401247F4D7F4B1B682246294631
S1130FB0002000F079FC7D4B1B6822462946012065
S1130FC000F072FC7A4C2146002000F06DFC2146B2
S1130FD0012000F069FC322002F0A8FEBDE8F88F81
S1130FE00120FFF72FFC842803D85F4D5F4C714E1E
S1130FF014E001235C4A13605C4A1360322002F05F
S113100095FE8FE70122594B1A60322002F08EFEC2
S113101088E7544B1B68B3F5FA7F26D22868FFF79C
S113102011FC8428EED82368002BF7D14D4B1B68A4
S1131030614A12689A42ECD04A4B19685E4A1160C0
S11310401A68A6FB02131B09322101FB1323002B90
S1131050DFD143210020FFF7FDFB43210120FFF7EF
S1131060F9FB2368002BD4D0D8E7DFF808B1594640
S1131070002000F019FCDFF800A15146002000F028
S113108013FCDFF8F890D9F800203D49002000F067
S11310900BFCDFF8F080D8F800203B49002000F07A
S11310A003FC3A4F3A683A49002000F0FDFB394E00
S11310B032683949002000F0F7FB384D2A783F495F
S11310C0002000F0F1FB3E4C374B1B680022214608
S11310D0104600F0E9FB5946012000F0E5FB5146BB
S11310E0012000F0E1FBD9F800202549012000F09F
S11310F0DBFBD8F800202449012000F0D5FB3A6836
S11311002349012000F0D0FB32682349012000F07C
S1131110CBFB2A782949012000F0C6FB234B1B682E
S113112001222146104600F0BFFB264C2146002038
S113113000F0BAFB2146012000F0B6FB0C4B1B6803
S11311405B68B3F1FF3F08D01F4C2146002000F03C
S1131150ABFB2146012000F0A7FB322002F0E6FDA4
S1131160BDE8F88FA0140020EC4E0020044F0020AE
S11311706407FF1F60660000C4660000E44E0020A0
S1131180E4660000DC4E002004670000D84E002016
S113119024670000E04E002044670000084F002050
S11311A0E8670000FC6700004C6900005869000013
S11311B0346800001F85EB516807FF1F6467000057
S11311C078670000A8670000706800002DE9F84304
S11311D0254A264B264813F8011F02F8011F8342B3
S11311E0F9D10022234B1A60234B1A68234B9A42ED
S11311F001D0BDE8F883204B1B7B012BF9D12027BC
S11312001C4EDFF88490DFF87C80306800F5BF2343
S113121003F2FF731A4D05F580512C4613F8012F84
S113122004F8012F8C42F9D100F50031C9F80010FF
S11312304FF48052404600F0A9F8336803F5805318
S11312403360013FE1D1FF2305F8013FAC42FBD1FC
S11312504FF480524FF4BE210A4800F097F800BFC3
S113126000BF00BFC5E700BFF34E0020FFEF05003D
S11312700FF00500E84E0020F44E002055AA5AA5B0
S11312800F4F0020104F00200C4F002070B5FFF7C7
S11312909DFFFFF727FE02F065FD322002F046FDB8
S11312A01F2002F043FD212002F040FD232002F024
S11312B03DFD0E4C2068FFF701FE02F045FD23685A
S11312C05E680B4D32462946002000F0EDFA094CC9
S11312D02146002000F0E8FA32462946012000F0B9
S11312E0E3FA2146012000F0DFFA70BD6407FF1F16
S11312F078680000B4680000024A537803F07F0362
S1131300537070470000024010B50A4C4FF0FF3391
S1131310A36100220849122002F0DCFC122002F032
S1131320F9FC02F011FD2146044802F019FB044BBC
S1131330188010BD78140020F9120000E86800003D
S113134094140020F8B507460D460A0BC1F30B03AD
S113135003B101320A4C0B4BA361120339462046F8
S113136002F064FB084E30804FF0FF33A361012389
S1131370C5F30F123946204602F0A4FB3080F8BDB5
S113138078140020D107FF1F941400202DE9F041A8
S113139082B080460E461746322002F0C7FC134C3A
S11313A0134BA3614FF480523146204602F03EFBBA
S11313B0104D28804FF0FF33A36143463A4631462F
S11313C0204602F0B5FB2880012301930A4B0093C9
S11313D043463A463146204602F006FC2880322035
S11313E002F098FC02B0BDE8F08100BF7814002040
S11313F0D107FF1F941400207414002008B54FF483
S11314000041034804F003F8002002F09BFA08BDF1
S1131410C0F00F4000B583B008230093144B154A65
S11314201549164802F0A4F81549164802F050F878
S11314301549164802F04CF81549164802F048F8C8
S11314401549164802F044F81549164802F040F8C8
S11314501549164802F03CF81549164802F038F8C8
S11314601549164802F034F803B05DF804FB00BFD8
S11314700069000020690000FC680000904D002015
S1131480E804FF1F304D0020F804FF1F404D0020EA
S11314900805FF1F504D00201805FF1F604D002058
S11314A02805FF1F704D00203805FF1F804D0020C8
S11314B0C804FF1F104D0020D804FF1F204D00203A
S11314C008B50023164A0121164801F01FFE012128
S11314D0002001F029FE0023134A0121134804F0DF
S11314E0B9FB0021012004F0CBFB11490A2003F0D1
S11314F07EFF00220F49162002F0ECFB162002F0BA
S113150015FC0D49002002F0EFF9FFF783FF00F00E
S113151051FA00F013F8FFF7F7FEFFF7AFFC08BD30
S11315200C4D00207C04FF1F6C4E00209806FF1F0A
S1131530A805FF1FFD1300004069000008B51C4901
S1131540002002F043FC1B4A0021084602F0F2FC92
S1131550194A0121002002F0EDFC184A0221002062
S113156002F0E8FC164A0321002002F0E3FC00220A
S11315701449302002F0AEFB00221349312002F05E
S1131580A9FB00221149322002F0A4FB00221049D9
S1131590332002F09FFB0421002002F06DFC0221A5
S11315A0322002F0E7FB322002F0B4FB08BD00BF9A
S11315B0486900004805FF1F6005FF1F7805FF1FED
S11315C09005FF1FED07FF1F3508FF1F1D08FF1FB4
S11315D00508FF1F022900D070470122014B1A7031
S11315E0FAE700BF0004FF1F022900D07047012260
S11315F0014B1A70FAE700BF0104FF1F022900D053
S113160070470122014B1A70FAE700BF0104FF1F63
S113161030B44268138804899C4207D8C368012205
S11316201A7001230B60406930BC70474469257807
S11316300469E55401331380F3E7000038B5044628
S113164090F82830002B43D1042913D0002941D12C
S1131650244B1B880122244B1A70244C4FF4006540
S11316602A46204604F0C9FB2A462146022003F0FC
S11316707FFB38BDC468CCB1C4F50064194B1B882A
S113168014FA83F3B3F5006F13D30122164B1A70C7
S1131690164C4FF400652A460021204604F0ADFBA9
S11316A02A462146022003F05DFA38BD4FF4006457
S11316B0E4E70C4D288822460C490D4B13FA80F0C0
S11316C004F090FB2B8814FA83F4A4B22C80DFE797
S11316D0012B00D038BD00F10C011046FFF798FF34
S11316E06060F7E7023D0020003D0020083D002037
S11316F00035002038B5044690F82830002B43D13B
S1131700042913D0002941D1244B1B880122244BE6
S11317101A70244C4FF400652A46204604F06DFBF1
S11317202A462146012003F023FB38BDC468CCB10E
S1131730C4F50064194B1B8814FA83F3B3F5006FE6
S113174013D30122164B1A70164C4FF400652A4627
S11317500021204604F051FB2A462146012003F0D3
S113176001FA38BD4FF40064E4E70C4D28882246A2
S11317700C490D4B13FA80F004F034FB2B8814FA57
S113178083F4A4B22C80DFE7012B00D038BD00F134
S11317900C011046FFF73CFF6060F7E7E22C0020E5
S11317A0E02C0020E82C0020E024002038B504467A
S11317B090F82830002B43D1042913D0002941D1BB
S11317C0244B1B880122244B1A70244C4FF40065CF
S11317D02A46204604F011FB2A462146002003F045
S11317E0C7FA38BDC468CCB1C4F50064194B1B8872
S11317F014FA83F3B3F5006F13D30122164B1A7056
S1131800164C4FF400652A460021204604F0F5FAF0
S11318102A462146002003F0A5F938BD4FF40064A0
S1131820E4E70C4D288822460C490D4B13FA80F04E
S113183004F0D8FA2B8814FA83F4A4B22C80DFE7DE
S1131840012B00D038BD00F10C011046FFF7E0FE7B
S11318506060F7E7C21C0020C01C0020C81C0020E8
S1131860C014002084B00346084A07CA0DF1100CC6
S11318700CE907000CEB830353F80C2C516800238C
S11318800B801268138004B0704700BF48660000E4
S113189000B583B002AB03F8011D0122194603F021
S11318A01FF903B05DF804FB0EB430B582B00546F1
S11318B005AA52F8041B01920B4804F0BFFAB0F5D4
S11318C0006F00D9FEE70446022D05D9204602B078
S11318D0BDE8304003B0704741F288330246024904
S11318E0284603F0CFF8F1E70C45002070B485B02A
S11318F003460D46124A07CA04AC04E9070004EB88
S1131900830353F80C4C66680E480F4933880380F0
S113191023681B880B80028892B20B889BB29A4280
S1131920F4D9094A13889BB22169CB5C2B702168D6
S1131930138801339BB213800B8005B070BC7047D1
S113194048660000084500200A450020F0B585B02F
S113195003460F4616460D4A07CA04AC04E90700BD
S113196004EB830353F80C5C6B681B882A681488A7
S1131970A342FDD9296932462144384604F032FA9B
S11319802B6834441C8005B0F0BD00BF48660000DD
S113199084B00346064A07CA0DF1100C0CE907008F
S11319A00CEB830353F80C3C5B68188804B0704755
S11319B04866000010B5464C22464649002003F014
S11319C05BF9454A4FF400631381444B5360444B25
S11319D01360444BD360444B5361444B13614449FB
S11319E0002003F03BF800224249104603F040F87F
S11319F0E379002B45D0012B4AD03F4C22463F4986
S1131A00012003F039F93E4A4FF4006313813D4B42
S1131A1053603D4B13603D4BD3603D4B53613D4B95
S1131A2013613D49012003F019F800223B490120CC
S1131A3003F01EF8E379002B30D0012B35D0384C5D
S1131A4022463849022003F017F9374A4FF400635D
S1131A501381364B5360364B1360364BD360364B91
S1131A605361364B13613649022002F0F7FF00221E
S1131A703449022002F0FCFFE379E3B1012B21D0C9
S1131A8010BD4FF400621849002003F06BF8B4E76E
S1131A9001221549002003F065F8AEE74FF4006217
S1131AA01B49012003F05EF8C9E7012218491046DA
S1131AB003F058F8C3E74FF400621F49022003F013
S1131AC051F810BD01221C49022003F04BF8D7E75E
S1131AD04C690000D04D0020A8140020C21C002036
S1131AE0C41C0020C01C0020C81C0020C0140020FE
S1131AF0AD170000D515000058690000044E002001
S1131B00C8240020E22C0020E42C0020E02C00203B
S1131B10E82C0020E0240020F5160000E915000060
S1131B2064690000384E0020E8340020023D0020A3
S1131B30043D0020003D0020083D00200035002029
S1131B403D160000FD1500004FF0E022D2F8883D5C
S1131B5043F47003C2F8883D064BA2F1DB62A2F5A0
S1131B60D7525A605A6842F220121A604FF6FF7236
S1131B709A60704700200540264B274A9A4208D0B5
S1131B8013462448254A13F8011B02F8011B984206
S1131B90F9D1234B234A9A4208D013462048224ABB
S1131BA013F8011B02F8011B8342F9D11F4B204A91
S1131BB09A4206D0134600211C4A03F8011B9342A3
S1131BC0FBD11C4B1C4A9A4208D0134619481B4AA5
S1131BD013F8011B02F8011B8342F9D1184B194A6F
S1131BE09A4212D010B4184CA40808D01946002305
S1131BF051F8040B42F8040B0133A342F8D1134B00
S1131C00104A1A605DF8044B7047104B0C4A1A6076
S1131C10704700BFD06F0000006C00000004FF1F7D
S1131C2090700000D06F0000D007FF1F205F0020DD
S1131C300000002090700000907000000000002060
S1131C40000000000000FF1F0004000008ED00E099
S1131C50074B5B69DBB2042B06D0802B06D0012B2B
S1131C600CBF0120042070470220704703207047F6
S1131C7000E00740044BD3F8003113F0807F1ABF13
S1131C80024B18680020704700400640904E002028
S1131C9010B584B00B4600293BD0444AD2F8002149
S1131CA012F0007F7DD1414AD2F8001121F40001E5
S1131CB0C2F800114FF08061C2F8001100213C4AC3
S1131CC01160002870D05A7A120202F4E062197A84
S1131CD001F007010A433548C0F80421DA791201FA
S1131CE002F030029979C90001F008010A435979D8
S1131CF0890001F004010A43C0F808211A79012A75
S1131D0029D0E2B1022A32D01A68294B1A60294C30
S1131D103BE000238DF804308DF80C3001228DF85F
S1131D2008208DF809208DF805208DF8063002234F
S1131D308DF8073004AB204A43F8102DADE71A7B29
S1131D40002A14BF4FF40002002242F00102174996
S1131D50C1F80021D8E71A7B002A14BF4FF400020F
S1131D60002242F001121149C1F80021CCE71A7B8C
S1131D70002A14BF4FF403024FF4403242F0010230
S1131D800A49C1F80021BFE7013CFFF773FF18B906
S1131D90002CF9D1032005E0002C14BF00200320FF
S1131DA000E0022004B010BD0020FBE70040064024
S1131DB0904E002088E7300000127A00084BD3F8D8
S1131DC0003213F0807F09D0054BD3F8083203F0BA
S1131DD00103002B034808BF002070470020704710
S1131DE00040064000127A0010B582B00B4600296C
S1131DF038D02D4AD2F8002212F0007F4FD12A4A5F
S1131E00D2F8001221F40001C2F800120021C2F835
S1131E100012002846D09A78120202F4E06259783F
S1131E2001F007010A432049C1F804221A7802F09C
S1131E300102C1F8082259799A791B79002B14BF41
S1131E4003230123002914BF042100210B43002A8A
S1131E5014BF4FF4000200221343134AC2F80032A5
S1131E60642410E000238DF8043001228DF805204D
S1131E708DF806308DF801208DF8022002AB03F8AE
S1131E80082DB6E7013CFFF799FF18B9002CF9D1EA
S1131E90032005E0002C14BF0020032000E00220F2
S1131EA002B010BD0020FBE700400640054BD3F80C
S1131EB0003313F0807F1DBF024BD3F80833024870
S1131EC00020704700400640006CDC0210B582B070
S1131ED00B46002932D0294AD2F8002312F0007FA1
S1131EE047D1264AD2F8001321F40001C2F80013A6
S1131EF04FF08061C2F8001300283DD09A78120296
S1131F0002F4E062597801F007010A431B49C1F861
S1131F1004231A7802F00302C1F808239A795B7942
S1131F20002B14BF01230923002A14BF4FF400021D
S1131F3000221343C1F8003364240EE001238DF81A
S1131F40053000228DF806208DF801308DF802301E
S1131F5002AB03F8082DBEE7013CFFF7A7FF18B951
S1131F60002CF9D1032005E0002C14BF002003202D
S1131F7000E0022002B010BD0020FBE70040064054
S1131F8008B50F4BD3F8003613F0807F02D100233D
S1131F90184608BDFFF76EFE03460028F8D008492E
S1131FA0D1F80826C2F302220132B0FBF2F3D1F8D1
S1131FB00826C2F30442103203FB02F35B08E7E78E
S1131FC00040064010B584B00C4699B13D4BD3F89F
S1131FD0003613F0007F72D13A4BD3F8002622F476
S1131FE00002C3F800264FF08062C3F80026A0B9AF
S1131FF0002065E000238DF804308DF80B300122B9
S11320008DF808208DF809208DF8053007228DF809
S113201006208DF8073001ACD8E7FFF72BFE637973
S11320201B0203F4E063227902F0070213432549FB
S1132030C1F8043663781B0203F4E063A278120447
S113204002F4F8121343C1F808362378012B16D092
S11320504BB1022B1FD04FF47A74FFF791FF48BBAA
S113206034B3013CF9E7E379002B14BF4FF40003C8
S1132070002343F00103134AC2F80036EBE7E37987
S1132080002B14BF4FF40003002343F001130D4A47
S1132090C2F80036DFE7E379002B14BF4FF40303E3
S11320A04FF4403343F00103064AC2F80036D2E746
S11320B0032005E0002C14BF0020032000E00220D0
S11320C004B010BD004006402DE9F04180460D46A5
S11320D08C7801344E7806FB04460F7807FB0447DE
S11320E0CB78013B052B1CD8DFE803F00312151B4A
S11320F01B18FFF7BFFD0009B8F1020F4AD0B8F171
S1132100030F7BD0B8F1010F0DD00020BDE8F081A2
S1132110FFF754FEEFE7FFF7C9FEECE7FFF730FFE8
S1132120E9E70020E7E7EA7802EB42015B4B53F86A
S113213021301B0904FB03F4A04200F293800B46F8
S1132140564901EB83035B681B0906FB03F6B042A7
S113215000F28B8002EB420301EB83039B681B09B3
S113216007FB03F7B84200F28380AB781B0403F447
S11321707023120602F0706213432A7802F00F02F1
S113218013436A781201D2B21343454A53610020C3
S1132190BDE8F081EA7802EB4201424B53F821306A
S11321A01B0904FB03F4A04265D80B463D4901EB2F
S11321B083035B681B0906FB03F6B0425ED802EB9F
S11321C0420301EB83039B681B0907FB03F7B84237
S11321D057D8AB781B0403F47023120602F0706224
S11321E013432A7802F00F0213436A781201D2B221
S11321F013432B4A93610020BDE8F081EB7803EB95
S11322004301294A52F82120120904FB02F4A04296
S11322103AD80A46244901EB82025268120906FBA5
S113222002F6B04233D803EB430201EB8202926818
S1132230120907FB02F7B8422CD8AA78120402F458
S113224070221B0603F0706313432A7802F00F0216
S113225013436A781201D2B21343114AD3610020A6
S1132260BDE8F0810120BDE8F0810120BDE8F081E6
S11322700120BDE8F0810120BDE8F0810120BDE826
S1132280F0810120BDE8F0810120BDE8F08101204A
S1132290BDE8F0810120BDE8F08100BF686A00005C
S11322A000400640BC6A0000146A000038B50546C8
S11322B0FFF7CEFC2946FFF707FF044658B9E87834
S11322C00A220849013A0B69C3F30363984204D014
S11322D0002AF7D10324204638BD002A08BF03246E
S11322E0F9E700BF0040064010B504461B4B1B69CC
S11322F0C3F30363013B052B1DD8DFE803F003138D
S1132300161C1C19FFF7B6FC144B1B69C3F30343DB
S11323100133B0FBF3F0012C0FD0ECB1022C14D03C
S1132320002010BDFFF74AFDEEE7FFF7BFFDEBE726
S1132330FFF726FEE8E70020E6E7084B1B69C3F336
S113234003130133B0FBF3F010BD044B1B6903F01E
S11323500F030133B0FBF3F010BD00BF0040064093
S113236008B50F4B1B6AC3F30363062B15D8DFE8CC
S113237003F004080B0E141411000220FFF7B4FF3D
S113238008BDFFF777FC08BDFFF718FD08BDFFF790
S11323908DFD08BDFFF7F4FD08BD002008BD00BF9A
S11323A00040064008B541B1012931D00020024661
S11323B010B1431E22FA03F008BD0438032852D892
S11323C0DFE800F00B02141DFFF770FD0246294BF5
S11323D0D3F8040300F00700EAE7FFF7EFFC024636
S11323E0244BD3F8040200F00700E1E7FFF742FCB6
S11323F00246204BD3F8040100F00700D8E7FFF7AA
S1132400BFFD02461B4BD3F8040600F00700CFE7DC
S1132410043803282AD8DFE800F00B02141DFFF764
S113242045FD0246134BD3F80403C0F30220BFE773
S1132430FFF7C4FC02460F4BD3F80402C0F302209A
S1132440B6E7FFF717FC02460A4BD3F80401C0F3C2
S11324500220ADE7FFF794FD0246064BD3F80406CD
S1132460C0F30220A4E700200246A1E700200246B0
S11324709EE700BF0040064008B5114B1B69C3F33B
S11324800113032B19D8DFE803F00207101300210E
S11324900620FFF787FF08BD094B186900F002000A
S11324A0002818BF4FF4FA4008BD064B186808BD51
S11324B000210520FFF776FF08BD002008BD00BFFE
S11324C000800440704E002038B51C4B33F81030A7
S11324D09B0003F1804303F5CA231D68C5F3C005BF
S11324E01C6804F00704AC4225D31868C0F380705C
S11324F010B31B68C3F30263013B052B19D8DFE853
S113250003F0030C101818140620FFF74BFF0134D6
S1132510B0FBF4F005FB000038BD0420FFF742FFD8
S1132520F5E70520FFF73EFFF1E70720FFF73AFF45
S1132530EDE70020EBE7002038BD00BF7069000024
S1132540114B1B69C3F38103022B07D0032B0ED05D
S1132550002B0CBF4FF4FA30002070470A4B186967
S113256000F00200002818BF4FF4FA407047064BF1
S1132570186910F0020006D0186900F00100002864
S113258018BF4FF47A7070470080044008B5244B9C
S11325905B6813F4006F40D0214B5B68C3F30313F3
S11325A00E2B09D8DFE803F00A080D081208171CDF
S11325B020252F0829082C00002026E0FFF7D0FE54
S11325C023E001210620FFF7EDFE1EE00121042097
S11325D0FFF7E8FE19E001210520FFF7E3FE14E010
S11325E00020FFF781FE10E001210720FFF7DAFE4B
S11325F00BE00120FFF778FE07E0FFF7A1FF04E0FE
S1132600FFF73AFF01E04FF4FA30054B5B68C3F380
S113261002230133B0FBF3F008BD002008BD00BF66
S113262000800440F0B5A1B028B304460646002853
S113263000F0FF80644B1B69C3F30363032B00F0BA
S1132640C980FFF733FC002800F0B48003238DF821
S1132650073000228DF8062001228DF8052020A8DD
S113266000F87C3DFFF722FE0546002800F0B2800A
S1132670284621B0F0BD01238DF80B3000228DF8DF
S11326800C208DF80D308DF80E208DF808308DF863
S113269009308DF80A308DF816308DF814308DF825
S11326A015208DF80F208DF810308DF811308DF82D
S11326B038300D928DF82530444906918DF81C2050
S11326C08DF824208DF81D308DF81E2002208DF801
S11326D01F008DF820308DF821308DF830308DF8C2
S11326E028208DF82F208DF829200C218DF82A1010
S11326F08DF82B208DF82C308DF82D308DF83D3051
S113270003218DF83C108DF84B308DF841108DF875
S113271040208DF83F308DF83E308DF845008DF81F
S113272044308DF843208DF8421006208DF849007E
S11327308DF848208DF847308DF8461024491E91B5
S113274022211D918DF84C308DF84D208DF84E20AE
S11327508DF84F208DF850308DF854308DF853306B
S11327608DF852208DF851208DF868308DF869303D
S11327708DF86A308DF86B308DF86C308DF86D30D3
S11327808DF873308DF858301792189219928DF88D
S11327906E308DF86F308DF870208DF871208DF8C3
S11327A072208DF87C308DF87D308DF87E2002AE5D
S11327B034463FE700210120FFF788FB0546002847
S11327C07FF456AF42E700BF0040064000127A0093
S11327D0A006FF1F3146E078FFF706FB05460028F8
S11327E000F02381FFF734FA022800F0588103280F
S11327F000F05881012800F03281002D7FF438AFB9
S113280094F8303013B1E26AA84B1A6094F835306A
S113281053B1A7490A6A22F0706294F834301B0657
S113282003F0706313430B6294F84330002B40F0C1
S1132830A68114F16C0F35D0236F002B32D0E36ED8
S113284083B300219B489C4D01EB8102236F9B5C69
S113285030F813309B0003F1804303F5CA231E684C
S113286026F080461E60236F9F189E5CBB781B0673
S113287003F0E063FA78D20002F0080213433A79D5
S113288002F0070213437A78002A14BF4FF0804203
S11328900022134330F8162045F822300131E36E4C
S11328A09942D1D394F84430C3B194F8463094F8A3
S11328B047208249496821F47F6194F84500002843
S11328C014BF4FF4006000201B01DBB2120202F4BB
S11328D0E06213430B430343784A536094F848304F
S11328E0DBB194F84A3094F849207449096921F01D
S11328F03F0194F84C00084394F84B10002914BF8E
S1132900022100219B0003F00C030343120102F097
S1132910300213430B43694A136194F86030002B6F
S113292037D0664B196C21F0010194F861200A43F9
S11329301A641B6C23F0020394F86220002A14BF6B
S11329400222002213435D4A1364136C23F0040330
S113295094F86320002A14BF042200221343574A28
S11329601364136C23F0080394F86420002A14BF42
S1132970082200221343514A1364136C23F01003FA
S113298094F86520002A14BF1022002213434B4AF6
S1132990136494F8503033B1494B626D1A60A26DE0
S11329A05A60E26D9A6094F86630EBB1434A936ED4
S11329B000209066516821F4805194F868301B031C
S11329C003F480530B435360906694F867305BB113
S11329D094F869305B0003F00E0394F86A2042F027
S11329E080521343354A936694F87430002B00F0F8
S11329F0E28034498B7803F07F0394F8752082F0E9
S1132A00010243EAC213DBB28B7094F97630002BD7
S1132A10BCBF20335BB22B490A7903F01F0302F0D9
S1132A20E00213430B71002522E604F11001607FDC
S1132A30FFF72EF9054600287FF4D4AE04F12001F7
S1132A4094F82800FFF7BEFA0546FFF701F90228BB
S1132A5025D0032826D0012801D0002601E004F166
S1132A603606002D7FF4C9AEF378032B2CD08DF8F5
S1132A700730B3788DF8063073788DF805303378E5
S1132A8020A800F87C3DFFF711FC054600287FF4E0
S1132A90B4AEE11DA07BFFF719FA0546ADE604F1DB
S1132AA03A06DEE704F13E06DBE700BF704E002085
S1132AB00040064070690000005006400080044059
S1132AC0744E002000D0074094F828300BBB637F7D
S1132AD093BBE378002B42D10125002D7FF48DAE0A
S1132AE0E11DA07BFFF7F2F9054600287FF485AECF
S1132AF0F3788DF80730B3788DF8063073788DF855
S1132B000530337820A800F87C3DFFF7CFFB05465D
S1132B1073E606238DF8073002238DF8063001236F
S1132B208DF8053020A800F87C3DFFF7BFFB054673
S1132B30637F7BB10128D0D101238DF807300022B7
S1132B408DF806208DF8053020A800F87C3DFFF7AD
S1132B50ADFB0546E378002BBFD0012DBDD1022388
S1132B608DF8073000238DF806308DF8053020A845
S1132B70012300F87C3DFFF799FB0546ADE704F11E
S1132B8036010120FFF7A0FA054600287FF470AD56
S1132B9004F13A010220FFF797FA054600287FF472
S1132BA067AD04F13E010320FFF78EFA05460028C5
S1132BB07FF45EAD3DE600255AE500BF70B50446DE
S1132BC00D46112807D9252840F285804F2840F268
S1132BD07781042070BD11287AD8DFE800F009134A
S1132BE0191F24292E33383C41484F565D646B72BB
S1132BF00020FFF779FB03460020002D00F0D2816E
S1132C002B6070BD0120FFF76FFB03460020F4E743
S1132C100220FFF769FB03460020EEE7FFF7B6FC4E
S1132C2003460020E9E7FFF7C9F803460020E4E77C
S1132C30FFF73CF903460020DFE7FFF71BF80346E4
S1132C400020DAE7FFF79CF903460020D5E7AD4BF7
S1132C501B680020D1E7FFF783FB03460020CCE785
S1132C6000210420FFF79EFB03460020C5E7012155
S1132C700420FFF797FB03460020BEE70021052050
S1132C80FFF790FB03460020B7E701210520FFF77B
S1132C9089FB03460020B0E700210620FFF782FBF2
S1132CA003460020A9E701210620FFF77BFB03462A
S1132CB00020A2E700210720FFF774FB0346002051
S1132CC09BE701210720FFF76DFB0346002094E7F3
S1132CD00023042091E7A0F11504102C00F2B98020
S1132CE0DFE804F00915212D38444F585D697984D3
S1132CF08C959EA7AF00844BDB68C3F30163022B62
S1132D0000F2AA80814A52F8233000203DE07E4B35
S1132D10DB68C3F38163022B00F2A1807B4A52F883
S1132D202330002031E0784BDB68C3F30173022BBE
S1132D3000F29880754A52F82330002025E0724B47
S1132D40DB689B0F022B00F29080704A52F823300C
S1132D5000201AE06C4BDB68C3F30143022B00F242
S1132D6087806A4A52F8233000200EE0664BDB6805
S1132D70C3F38143022B7ED8644A52F823300020E7
S1132D8003E0FFF703FC03460020002D00F00A8156
S1132D902B6070BDFFF770FB03460020F5E75C4B2A
S1132DA09B78DB0902D000231846EEE7FFF7C8FB47
S1132DB003460020E9E7564B9B78DB095ED1524B72
S1132DC01B6913F002035CD04F4B1B6913F0010322
S1132DD059D10020D9E74E4B9B78DB0957D14A4B98
S1132DE01B6913F0020355D10020CEE7484B9B78B2
S1132DF0DB0953D14FF4FA330020C6E7424B1B6C76
S1132E00C3F30013002B4CD14FF48070BDE73E4B4D
S1132E101B6CC3F3C003002B46D14FF48070B4E79E
S1132E20394B1B6CC3F38003002B40D14FF48070EB
S1132E30ABE7354B1B6CC3F34003DBBB4FF4807033
S1132E40A3E7314B1B6C13F0010336D14FF48070B0
S1132E509BE70023042098E70023184695E7002306
S1132E60184692E7002318468FE7002318468CE79C
S1132E700023184689E70023184686E700231846EE
S1132E8083E7002081E74FF47A7300207DE7002375
S1132E9018467AE74FF4FA43002076E700231846F1
S1132EA073E70023184670E7002318466DE70023F4
S1132EB018466AE70023184667E70023184664E7C4
S1132EC0262805D804200023002D6BD02B6070BD6C
S1132ED0A0F13303DBB21C2B07D80E4A22FA03F30A
S1132EE013F0010F18BF0420EDD10B4B33F814205D
S1132EF00A4B53F8223013F0804F42D14FF48070C4
S1132F00E1E700BF704E002000800440744E0020B2
S1132F1000D0074041810010706900000050064055
S1132F200120FFF7E1F9B8BB00234FF48070CBE731
S1132F300020FFF7D9F90028F6D02DE00220FFF792
S1132F40D3F90028F0D027E016F0080F06D116F0C8
S1132F50100F0BD100234FF48070B5E700212046F9
S1132F60FFF7B2FA034616F0100F04D001212046F1
S1132F70FFF7AAFA0346002B14BF00204FF4807019
S1132F80A2E7094B1E5D16F0200FC9D116F0400FC1
S1132F90CED116F0800FD1D116F0180FD4D1002362
S1132FA0184691E770BD00BF106B000070B582B089
S1132FB005460C46FEF74CFE06469DB12B68022BD7
S1132FC00ED0042B10D0012B0CBF012504256CB1AD
S1132FD02378043B032B4AD8DFE803F04B434547EF
S1132FE00225F4E70546F2E70325F0E7FEF75EFF66
S1132FF058B103238DF8073000228DF806200122F2
S11330008DF805208DF8043043E0FEF7B9FF58B180
S113301006238DF8073002238DF8063001238DF83E
S113302005308DF8043034E0FEF724FE50B101235E
S11330308DF8073000228DF806208DF805308DF8C4
S1133040043026E0FEF7BAFE18B302238DF80730E9
S113305000238DF806308DF8053001238DF80430F7
S113306017E0032306E0012304E0062302E0FF2324
S113307000E002238DF807300C4B62889A5C8DF8CF
S11330800620A2889A5C8DF80520E2889B5C8DF866
S11330900430B54205D001A92846FFF715F802B05F
S11330A070BD01A8FFF702F9F9E700BF646B0000E7
S11330B0154B1B69C3F30363013B052B20D8DFE8E1
S11330C003F00316191F1F1C062303700E4A13690D
S11330D0C3F30343013343801369C3F3031301337D
S11330E08380136903F00F030133C3807047042303
S11330F00370EBE705230370E8E707230370E5E7B4
S113310004230370E2E700BF0040064010B4054CFE
S113311020602171A2602373637300205DF8044B67
S1133120704700BF804E0020F0B583B007460E46BE
S11331308DF804008DF8051000F014FE334B1C7B51
S11331405C7301238DF80630002C4AD000242F4DE7
S113315004E00134E4B22B7BA34242D9AB6853F8B8
S11331602430002BF5D01A79022AF2D01A68996813
S113317001A890470028ECD06C73002EE9D140F2EE
S1133180031500238DF80630A400204E20E00134FE
S1133190E4B23B7BA34212D9BB6853F82430002B22
S11331A0F5D01A79012AF2D01A68996801A89047D3
S11331B00028ECD07C73002EE9D14FF4827500F026
S11331C0C3FD284603B0F0BD043C14F1040FF6D04F
S11331D0B3681B59002BF7D01A68996801A8904767
S11331E0F2E70A4D2B6853F82700FFF71BFA6F71BB
S11331F005460028C5D102238DF80630034B1B7BFE
S1133200002BDCD00024014FC6E700BF804E002015
S113321008B5FFF7D3FC08BD29B14118002300F815
S1133220013B8142FBD1704710B4064B1B6853F835
S11332302040616053F820309A6000205DF8044B10
S1133240704700BF944E002008B5084B1B6853F824
S1133250203000F00F00064A1077D07723B15A6867
S113326012B1197B9868904708BD00BF944E0020A6
S11332700080004038B5054600F00F0400222146C6
S1133280094800F000FA094B1B6853F8253053B184
S1133290054A1477D477947701221A735A6812B1C5
S11332A0197B9868904738BD00800040944E0020F8
S11332B02DE9F04F87B09DF84070119D0124BC406A
S11332C05FFA84FCB5FBFCF60CFB1656002E14BF0B
S11332D04FF0010A4FF0000A03D0504607B0BDE892
S11332E0F08F059304920391804600F00F06DFF8F7
S11332F000913146484600F0CBF9D9F8003043F04C
S11333008003C9F80030730103F1804202F5004BD9
S113331002F51042049810604B4441F210020598E3
S113332098500197009700231A463146484600F00A
S1133330E5F9039B032B12D8DFE803F0022D3D4C83
S1133340002241F204032BF8032064B2A4B27301F7
S113335003F1804303F5004341F214029C52244CD0
S11333602A463146204600F0E1F901223146204642
S113337000F00AFA04EB461641F21C02B35A1BB2DF
S113338043F002039BB2B3521A4B1B6853F8283024
S113339000221A73A1E764B2A4B241F204032BF829
S11333A00340730103F1804303F50043002141F21C
S11333B014029952D3E764B2A4B241F204032BF885
S11333C00340730103F1804303F5004341F2140207
S11333D09C52C4E7002241F204032BF8032073013A
S11333E003F1804303F5004341F214015A52B6E756
S11333F000800040944E002070B582B00446079DC2
S113340001959DF818500095FFF752FF054610B13D
S1133410284602B070BD04F00F040F4E089A2146EE
S1133420304600F0B1F906EB441641F21C03F35A9E
S113343023F008031B041B0C9DF82420002A14BF4E
S1133440082200221343640104F1804404F500447B
S113345041F21C02A352DBE70080004008B50122C0
S113346000F00F01024800F00EF9002008BD00BF73
S11334700080004008B5002200F00F01024800F06F
S113348002F9002008BD00BF0080004010B40F4BBB
S11334901C5C04F07F041C541C5C01F03F0104F02C
S11334A0C004214319541B5C03F0BF03002A14BF5A
S11334B0402200221A43054B1A541A5C42F080023F
S11334C01A5400205DF8044B704700BF00100240FE
S11334D02DE9F04180460C464D7805F00F06102189
S11334E0FFF79AFE227BA1786078FFF7CFFF0746AB
S11334F031461D4800F0CCF817B13846BDE8F081DC
S11335001A4B1B6843F8258053F82520157053F88F
S1133510253000221A73144D01223146284600F04A
S1133520ADF82B6813F0040F11D12378FF2B0ED0C4
S113353086F0030606F1804606F5004696F800215B
S113354003F00F0302F0F002134386F800316568BC
S1133550A1686278054B1B6853F82200456053F854
S113356022309960C9E700BF00800040944E0020DB
S11335702DE9F0420D4616469946069F244B1860E5
S11335804021FFF749FE234C204600F0A6F82268AC
S113359022F004022B789B0003F0040313432360FE
S11335A0236823F010036A78002A14BF1022002233
S11335B013432360102000F0ADFB174DAC1E1E35E5
S11335C034F9020F00F0A6FBAC42F9D1134800F025
S11335D020F9DEB1B9F1000F14D0AFB1043EA9F166
S11335E0040900252C4659F8041F56F8040FFFF768
S11335F06FFF002818BF05460134A742F3D12846BF
S1133600BDE8F0820025FAE70025F8E70025F6E793
S1133610944E002000800040786B000000100240AF
S113362000F00F0080304001014B1950704700BF7B
S11336300080004000F00F00400100F1804000F5E0
S1133640004041F21003C1507047000008B50A461B
S113365000F00F01014800F097F808BD0080004019
S113366008B500F00F01024800F0BDF808BD00BF26
S11336700080004000487047008000400AB901768D
S11336807047417670470AB981767047C1767047B2
S113369000EB4111002341F208028B5001F58052E6
S11336A0136041F204028B5241F206028B5241F242
S11336B00C028B5041F210028B5041F214028B52D7
S11336C041F216028B5241F218028B5041F21C0255
S11336D08B5241F21E028B52704738B5054603687F
S11336E023F4403323F0C60303600024E1B22846E8
S11336F0FFF7CEFF0134102CF8D138BD10B4DB0035
S1133700DCB29DF8083003F00703234343EAC223E5
S11337109DF80420120202F4E06213439BB280314C
S113372000EB4111CB805DF8044B7047036813F044
S1133730800F13D010B400EB411341F208041B595D
S1133740002B11DB00EB41131B5913F0804F0BD1FD
S113375022F0404200EB4110025112E000EB411014
S113376041F20803C250704700EB411041F20801D6
S1133770435823F47F7323F00303C2F309021A436B
S113378042505DF8044B704710B400EB411441F211
S11337901E03E35A13F4004F14D100EB411141F21C
S11337A01E000B5AC2F30E0203F4004313430B52E0
S11337B041F216000B5A03F400431A430A525DF80F
S11337C0044B704741F21E00235AC2F3080203F46B
S11337D07E431343235241F21600235A03F47E43DB
S11337E01A432252EBE700EB411241F21E03D35A73
S11337F013F4004F07D100EB411041F21603C05AF5
S1133800C0F30E00704741F21603D05AC0F308000B
S1133810704700231A46C2540133102BFBD1704762
S113382008B50020FFF710FD08BD08B50120FFF71B
S11338300BFD08BD08B50220FFF706FD08BD08B55D
S11338400320FFF701FD08BD08B50420FFF7FCFCC9
S113385008BD08B50520FFF7F7FC08BD08B506202C
S1133860FFF7F2FC08BD08B50720FFF7EDFC08BD23
S113387008B50820FFF7E8FC08BD08B50920FFF7E4
S1133880E3FC08BD08B50A20FFF7DEFC08BD08B557
S11338900B20FFF7D9FC08BD08B50C20FFF7D4FCBA
S11338A008BD08B50D20FFF7CFFC08BD08B50E20F4
S11338B0FFF7CAFC08BD08B50F20FFF7C5FC08BD1B
S11338C038B50020FFF7D6FEC56A002404E06D0871
S11338D00134E4B2102C06D015F0010FF7D02046C5
S11338E0FFF7C8FCF3E738BD154B1B7813F0010F45
S11338F020D10B79CA789A421ED2FF2B1ED08A7827
S11339000F4B5A710A79DA70CA789A704B78002B87
S113391014BF092301230A78012A05D0022A06D0FC
S1133920074A13700020704743F00403F8E743F09C
S11339300603F5E701207047012070470120704716
S11339400010064008B500F00DFA044BB4225A707A
S11339502C225A7000F0F8F908BD00BF0010064090
S113396003680B6043684B6083688B60C3680B61BA
S113397003698B612C4BDB6CC3F303330F2B4DD8E2
S1133980DFE803F0080F13171E2125292D303438E2
S11339903C4044484FF48033CB6000234B6100200B
S11339A070474FF0FF33CB60F7E74FF0FF33CB6046
S11339B0F3E74FF40043CB604FF480534B61EEE7E1
S11339C00023CB60F8E74FF0FF33CB60E5E74FF01F
S11339D0FF33CB60E1E74FF0FF33CB60DDE700233B
S11339E0CB60E9E74FF0FF33CB60D6E74FF4804379
S11339F0CB60E1E74FF40043CB60DDE74FF4803365
S1133A00CB60CAE74FF0FF33CB60C6E74FF0FF331C
S1133A10CB60C2E74FF48033CB60BEE7CB68B3F52D
S1133A20803FC9D3B9E700BF008004402DE9F047C7
S1133A300646174684688C4214D8C36823449942C6
S1133A4010D201F500010C1B4FF4006808F1FF339C
S1133A503B4214BF01200020194D4FF0700A4FF073
S1133A6009091CE03468A14224D3736823449942B1
S1133A7023D20C1B4FF48058E8E785F800A085F8A2
S1133A800790C4F30743AB71C4F307236B71E3B22C
S1133A902B71304603F0ACF8A7EB080744443FB160
S1133AA020B92B7813F0800FE7D10220BDE8F0870E
S1133AB0BDE8F0870120BDE8F0870120BDE8F0876C
S1133AC00000024038B584688C420DD8C56825448E
S1133AD0A94209D201F50001091B144C247814F001
S1133AE0800F0AD1022038BD0468A1421AD3456868
S1133AF02544A94218D2091BEFE70C4C7025257008
S1133B000125E571C1F30745A571C1F30725657169
S1133B10C9B22171110AE172D2B2A272637203F0C6
S1133B2067F838BD012038BD012038BD00000240CF
S1133B3012F0070F4ED12DE9F04781460C46154689
S1133B4082688A4208D8C16811448C4204D204F5C0
S1133B500004A41A00200CE0D9F80020944207D3F2
S1133B60D9F8041011448C4213D2A41A002000E0A6
S1133B7001205E1EDFF86C804FF0700A174F5DB3B2
S1133B8050BB98F8003013F0800F04D10220BDE838
S1133B90F0870120EDE788F800A0072388F80730B4
S1133BA0C4F3074388F80630C4F3072388F80530C4
S1133BB0E3B288F804303346094A13F8011F02F8C7
S1133BC0011FBA42F9D1484603F012F80834083DFF
S1133BD00836D4E701207047BDE8F0870F000240A3
S1133BE007000240000002402DE9F04F83B001932A
S1133BF09DF8349012F0030F04D00123184603B04B
S1133C00BDE8F08F064615468768B94219D3C368E4
S1133C103B44994215D201F50004E41B4FF0000A1D
S1133C205346DFF8A880DFF8A8B035B12BB998F86F
S1133C30003013F0800F0DD102230C9AC2F800A0BB
S1133C40DCE73768B94235D373683B44994235D2CF
S1133C50CC1BE3E7702388F80030022388F8073090
S1133C60C4F3074388F80630C4F3072388F8053003
S1133C70E3B288F8043088F80B90019B5A1E114B6C
S1133C8012F8011F03F8011F5B45F9D1304602F019
S1133C90AFFF034640B10C4A944286BFA7F5000A21
S1133CA0A24407EB040AC0E7043D019A04320192DE
S1133CB00434BAE74FF0000A0123BEE74FF0000ACC
S1133CC00123BAE70B000240FFFF7F00000002401F
S1133CD00F00024010B40B4B0B4C9C420DD02AB188
S1133CE000F11003084C54F8233013601030064BD5
S1133CF043F820105DF8044B7047044B044C9C427D
S1133D00F8D1ECE7000000000000FF1FD06F0000B6
S1133D10006C0000420900F01F00012303FA00F0C8
S1133D20014B43F82200704700E100E0430900F032
S1133D301F00012202FA00F02033024A42F8230055
S1133D40704700BF00E100E0054B1B68002B04DD59
S1133D50013B034A1360002B00DD704762B6FCE7A9
S1133D60984E002072B6024A1368013313607047FC
S1133D70984E0020002808DB0901C9B200F1604018
S1133D8000F5614080F80013704780B2C0F38102EF
S1133D90012A0DD010B40A4C0A4B022A18BF23463C
S1133DA000F003000901C9B219545DF8044B7047CF
S1133DB0054B00F003000901C9B21954704700BF54
S1133DC020ED00E01CED00E018ED00E070B582B0DD
S1133DD006460C46264D05EB80014720FFF718FAEE
S1133DE0002002A941F8040DFFF712FA55F8262025
S1133DF0019B03EB5203B3FBF2F213461D488168A7
S1133E0041F0020181602AB1013B00BF00BF00BF45
S1133E10002BF9D117498B6823F002038B601346FA
S1133E20886840F0010088602AB1013B00BF00BFF0
S1133E3000BF002BF9D121780E4B9A6822F00802BA
S1133E409A609A68002914BF082300231A43094B77
S1133E509A6061789A6822F004029A609B6800294B
S1133E6014BF042200221343024A936002B070BDBF
S1133E709C4E002000700340024A5369194351616B
S1133E80704700BF00700340F8B506460C4617465D
S1133E90244D05EB80014720FFF7BAF955F82600B9
S1133EA0214A0023A0FB0701FCF7D8FA10F1FF36E2
S1133EB041F1FF37230103F1804303F55C339B6A2F
S1133EC0C3F38103012B20D0022B24D1012F08BF7F
S1133ED0002E12D30120F8BD144A0023BB4208BFB0
S1133EE0B24210D3002F08BFB6F5803F05D3B0F11E
S1133EF0011006044FF6FF721643023424010C4BE2
S1133F001E510020F8BD0120F8BD012F08BF002E6E
S1133F10E2D30120F8BD012F08BF002EEDD301200C
S1133F20F8BD00BF9C4E002040420F00FEFF010080
S1133F300070034030B583B03023ADF80030312336
S1133F40ADF802303223ADF804303323ADF8063037
S1133F500D4659B9D37C002B40F0AE80574B996A7B
S1133F6021F002019962996A00230EE0D47C0B01CE
S1133F7003F1804303F55C33996A21F002019962ED
S1133F80996A002C14BF02230023144619432B0101
S1133F9003F1804303F55C3399621278996A21F046
S1133FA00C019962996A920002F00C020A439A6227
S1133FB06378012B69D06168AB1C1B013F4AD15067
S1133FC0227A2B0103F1804303F55C33996A21F4CF
S1133FD000019962996AD20502F400020A439A62C6
S1133FE0E268996A21F070619962996A120602F096
S1133FF070620A439A62217C9A6A22F480229A624D
S11340009A6A002914BF4FF4802300231A432B011A
S113401003F1804303F55C339A62617C9A6A22F46B
S113402000329A629A6A002914BF4FF400330023C5
S11340301A432B0103F1804303F55C339A62A17C9C
S11340409A6A22F480329A629A6A002914BF4FF461
S1134050803300231A432B0103F1804303F55C33BF
S11340609A62237DCBB915490B690122AA4023EA40
S113407002030B6102AB03EB450535F9080CFFF7AE
S113408055FE0023184603B030BD62682946FFF789
S1134090FBFE03460028F5D192E7084A1169012383
S11340A0AB400B43136102AB03EB450535F9080C38
S11340B0FFF730FE0023E5E70123E3E70070034048
S11340C0014BD960DB68704700700340036943EA21
S11340D0422242EA012202617047B1F57C5F07D0B7
S11340E04269012303FA01F1114341610020704741
S11340F0436943F47C534361F8E708B5002000F0BA
S1134100B5F808BD08B5012000F0B0F808BD08B541
S1134110022000F0ABF808BD38B51B4B53F8205013
S11341201A4B53F8204000232B7395F82430D3B94D
S1134130E36923F00203E361E36923F00103E3612C
S113414000F048F9A36923F48063A3610A2120469F
S1134150FFF7C3FF6B797BB9AB6A1BB1EA6A002135
S11341602846984738BDA36923F00203A361A369D5
S113417023F00103A361E3E705F1250001F002FE4A
S113418000236B71E8E700BFA04E00204C07FF1F1F
S113419010B5084B53F82040FFF7BEFF012211462B
S11341A02046FFF793FF012211462046FFF78EFFBA
S11341B0002010BD4C07FF1F70B50546294B53F86E
S11341C02060294B53F82040636913F4006F0BD02F
S11341D033694BB1FFF7DCFF0B212046FFF77DFF6E
S11341E0012386F8263070BD636913F4805F0CD018
S11341F0736953B12846FFF7CBFF0C212046FFF724
S11342006CFF022386F8263070BD636913F0020F39
S113421002D0738B9BB2CBB9636913F0010F02D048
S1134220338B9BB2B3B9338B9BB273B9A36923F0BD
S11342300103A361A36943F48063A361738B9BB2FD
S11342401BB9636913F4806F08D170BD284600F070
S11342507BF8E1E7284600F01DF8E4E72846FFF77D
S11342605BFFF2E7A04E00204C07FF1F02280DD889
S113427008B5074B53F820305B6A13F0010F02D1E5
S113428000F0FAF808BDFFF797FF08BD704700BFBC
S11342904C07FF1F2A4B53F820302A4A52F82000BB
S11342A0C26D02F0070293F82110891A11F0FF0180
S11342B045D0F0B504244FF0000C1FE0026E22F448
S11342C08012026600221A83F0BD12F8015B1A61A3
S11342D0B3F81CE017FA8EFE9EFBF6F206FB12E61C
S11342E0B6B29E8345661A8BD21B92B21A831A8B7E
S11342F092B21AB3013911F0FF011FD01A791AB121
S11343001A8B92B2012AD9D05E889A8B92B2B21AD1
S1134310042ADDBF9A8BB21A97B227461A695AB19A
S1134320012ED2D0022E03D052F8045B1A61CFE7DB
S113433032F8025B1A61CBE76546D3E7F0BD7047FC
S1134340A04E00204C07FF1FF0B4204B53F8201060
S11343501F4B53F82070FE6DC6F30246002E32D078
S11343604FF0040C22E0644600234869DA0025FA81
S113437002F202704A6901324A6101339AB29442EC
S1134380F3D8CB8B14FA83F2488892FBF0F300FB4A
S113439013239BB2CB834B8B1C1BA4B24C834B8B40
S11343A09BB283B1013E16F0FF060CD07D6F4C88A2
S11343B0CB8B9BB2E31A042BD5DCCB8BE41AA4B2CF
S11343C0002CD1D1DDE7F0BC704700BFA04E002027
S11343D04C07FF1F10B50A4B53F82040A36923F480
S11343E00063A361A36923F48053A3610B212046D6
S11343F0FFF773FE0C212046FFF76FFE10BD00BFD0
S11344004C07FF1F38B51A4B53F82040194B53F88B
S1134410205095F82430012B19D0E36923F00203CE
S1134420E361E36923F00103E361FFF7D3FF0023B2
S11344302B73012211462046FFF748FE0122114644
S11344402046FFF743FE6B7953B9002038BDA369BA
S113445023F00103A361A36923F00203A361E4E74A
S113446005F1250001F08EFC00236B71EDE700BF20
S11344704C07FF1FA04E002070B50646314B53F881
S11344802050314B53F820406B6913F4006F07D070
S113449023692BB1FFF7B6FF012384F8263070BDE2
S11344A06B6913F4805F08D0636933B13046FFF75A
S11344B0A9FF022384F8263070BD6B6913F0020F44
S11344C003D0638B9BB2002B2DD16B6913F0010FCA
S11344D002D0238B9BB253BB238B9BB21BB9AB691A
S11344E023F00103AB61638B9BB21BB9AB6923F06F
S11344F00203AB61638B9BB2A3B9238B9BB28BB9D1
S1134500AB6923F40063AB61AB6923F48053AB6103
S1134510A36A1BB1E26A002120469847637953B924
S11345200023237370BD3046FFF70EFFCDE73046FE
S1134530FFF7B0FED0E704F1250001F023FC0023CF
S11345406371EDE74C07FF1FA04E002010B50F4B21
S113455053F820301C7C0CB1022010BD0C4C54F8D4
S1134560200019609A6001221A740222DA85836994
S113457043F400238361836913F4002FFBD00122E9
S1134580044900F0ECFD002010BD00BFAC4E00203B
S1134590986B000017000300F0B585B01B4B53F86F
S11345A02040237C13B1022005B0F0BD13460A4617
S11345B00646174951F8205022600027A7600121C0
S11345C021740220E08594F82A000391029301915A
S11345D0009705F11C03FEF70FFF32460D4994F8CE
S11345E02A00FEF721FE94F82A00FEF737FFAB6994
S11345F043F40023AB61AB6913F4002FFBD02B69A8
S113460043F400032B610020CEE700BFAC4E002032
S1134610986B0000E146000038B5144B53F8204075
S1134620134B53F82050EB8D9BB2022B16D0002273
S11346301049204600F093FD00220F49204600F067
S11346408EFDA36923F40023A361A36913F4002F4F
S1134650FBD100232B74AB7C1BB938BD0023EB8545
S1134660EAE705F12C0001F08DFBF6E7986B0000FA
S1134670AC4E0020170003001600030038B5154B9C
S113468053F82040144B53F82050236923F40003BB
S1134690236195F82A00FEF7EDFE00220F4920461B
S11346A000F05DFDA36923F40023A361A36913F45F
S11346B0002FFBD1AB7C43B9EB8D9BB2022B04BF23
S11346C00023EB8500232B7438BD05F12C0001F089
S11346D059FBF1E7986B0000AC4E00201600030074
S11346E038B5194B53F82040184B53F82050012982
S11346F00DD0236A1BB1626A012120469847A36842
S11347008BB901221249284600F029FD38BD012346
S1134710E385FFF7B3FF236A002BF7D0626A032116
S11347202046984738BD216894F82A00FEF778FFA0
S1134730A16894F82A00FEF789FF0023A36094F887
S11347402A00FEF78BFE38BDAC4E0020986B0000AB
S11347501600030008B50E4B53F820300D4A52F8EA
S113476020001A681B7D43B1012B09D013785178BE
S113477043EA012100F0CAFC08BD1378037708BDA1
S11347801378517843EA012100F0B5FC08BD00BF5D
S1134790AC4E0020986B000010B5114B53F820303C
S11347A05C7C0CB1022010BD0E4C54F8204001205A
S11347B058745960DA6002221A86A36943F480238C
S11347C0A361A36913F4802FFBD00121204600F0DC
S11347D0DFFD01220449204600F0C1FC002010BD89
S11347E0AC4E0020986B0000150003002DE9F04347
S11347F085B0244C54F820506C7C1CB1022005B0C8
S1134800BDE8F0830F4606461F4B53F8204095F849
S113481029004FF00108CDF80C800292CDF80480F5
S11348204FF00009CDF800900B4604F11C024946F4
S1134830FEF7E2FD3246154995F82900FEF7F4FC2F
S113484095F82900FEF70AFE6F60C5F80C9085F80C
S1134850118002232B86A36943F48023A361A369F7
S113486013F4802FFBD00021204600F091FD01229B
S11348700749204600F073FC236943F400132361C5
S11348800020BCE7AC4E0020986B00005D4900009E
S11348901400030038B5154B53F82050144B53F84B
S11348A02040A36923F48023A361A36913F4802F18
S11348B0FBD10021204600F06BFDE36900220D4985
S11348C0204600F04CFCEB7C43B900236B742B8E28
S11348D09BB2022B04BF00232B8638BD05F12B00AD
S11348E001F050FA0023EB74EFE700BFAC4E002058
S11348F0986B00001500030038B5164B53F82040A0
S1134900154B53F82050A36923F48023A361A369B2
S113491013F4802FFBD10021204600F039FD2369D8
S113492023F400132361E36995F82900FEF7A2FD3F
S1134930EB7C43B92B8E9BB2022B04BF00232B8646
S113494000236B7438BD05F12B0001F01BFA002322
S1134950EB74EFE7986B0000AC4E002070B5054691
S1134960254B53F82040254B53F82060012904D0EF
S1134970238E9BB2022B13D070BD01232386FFF735
S1134980BBFFA3691BB1E269032120469847736901
S113499023F0C02323F4F81343F470237361E7E78F
S11349A0A3691BB1E269002120469847E3688BB9EB
S11349B02846FFF7A1FFA3691BB1E2690221204643
S11349C09847736923F0C02323F4F81343F4702346
S11349D07361D1E7616894F82900FEF72BFEE16862
S11349E094F82900FEF732FE0023E36094F82900CE
S11349F0FEF734FD70BD00BFAC4E0020986B000084
S1134A0010B582B0134B53F82030134A52F82000EB
S1134A105C681B7D73B1012B0FD00DF1060100F012
S1134A208FFBBDF806302370BDF806301B0A637097
S1134A3002B010BDC3692370FAE70DF1060100F05E
S1134A4076FBBDF806302370BDF806301B0A637090
S1134A50EEE700BFAC4E0020986B0000034B53F808
S1134A60203098699961DA61704700BFAC4E00202C
S1134A70034B53F82030186A19625A62704700BF1A
S1134A80AC4E002070B505461E46144B53F820402A
S1134A900123A37494F82830012B05D0FFF77CFD83
S1134AA028B1E08D80B270BDFFF750FDF8E73146C4
S1134AB004F12C0001F02CF90328F2D10023A37493
S1134AC00323E38594F82830012B03D02846FFF70D
S1134AD0D5FDE6E72846FFF79FFDE2E7AC4E002050
S1134AE02DE9F8431C4B53F8208098F8103013B18B
S1134AF00220BDE8F88381460F461646174B53F84B
S1134B002040A36943F40023A361A36913F4002F95
S1134B10FBD0B6B1124D02E00237023E8EB12946F7
S1134B20204600F079FB0028F9D0C8F80070484608
S1134B30FFF710FE98F81430002BEDD10137013E39
S1134B40ECE7A36923F40023A361A36913F4002F02
S1134B50FBD10020BDE8F883AC4E0020986B000028
S1134B601700020010B5074B53F820300024DC7402
S1134B7093F82830012B02D0FFF738FE10BDFFF761
S1134B800BFE10BDAC4E0020384B53F820303BB127
S1134B901A7C0AB1022070475B7C0BB1022070477B
S1134BA02DE9F04182B00C46314B53F8205001A955
S1134BB0304B185CFEF72CFB01984FEA840CB0FBD9
S1134BC0FCFC1FFA8CFC4FEA8C07B0FBF7F7BC42E5
S1134BD034BF3F1BE71BB0FBF4F8B8F1200F28BF2C
S1134BE04FF02008B8F1040F38D905264FF0040E11
S1134BF0324604E0013292B21646424513D806FB0F
S1134C0004F1B0FBF1F18BB202FB03F3B0FBF3F35D
S1134C109C4234BF1B1BE31ABB42EBD81FFA81FC36
S1134C201F46B646E6E7BEF1070F19D92A6922F0F6
S1134C30F8520EF1FF331B0603F0F85313432B61B4
S1134C402B6923F4FF5323F01F03CCF30C0C4CEA21
S1134C5003032B61002002B0BDE8F0814FF0040E85
S1134C602B6943F400332B61E0E700BFAC4E002016
S1134C70986B0000A46B0000F0B583B007460C46A7
S1134C801646364B53F8205001A9354B185CFEF7F5
S1134C90BFFA631E04F13301002203F8012F8B4293
S1134CA0FBD1304B43F82740F37984F82830B379AB
S1134CB02375337A84F82930737A84F82A302846A5
S1134CC000F0E0F931683846FFF75EFF3379002BD6
S1134CD03BD00122B179284600F0E6F93179284623
S1134CE000F0FAF92B69727923F4005343EA423352
S1134CF02B61AB6923F4E06343F44073AB61AB69AC
S1134D0043F00403AB610025E5852586294604F1BB
S1134D102B0001F04AF80646294604F12C0001F064
S1134D2044F8012E17D001280DD00F4B33F917404A
S1134D302A460E4B53F827102046FEF7CBFF204699
S1134D40FEF7E8FF284603B0F0BD0022B1792846FB
S1134D5000F0AAF9C2E73046F5E700BF986B0000FF
S1134D60A46B0000AC4E0020A86B00005807FF1F86
S1134D70034B53F820305960DA600020704700BFBD
S1134D80AC4E0020F8B506469D4B53F820409D4993
S1134D90204600F01CFA002836D19B4B53F82650CD
S1134DA09A49204600F038FA002850D040F20163B6
S1134DB02B8695F82830012B45D03046FFF79CFD13
S1134DC0AB691BB1EA69032128469847636923F05C
S1134DD0C02323F4F81343F4702363618C49204601
S1134DE000F0F5F9002840F09B808A49204600F045
S1134DF0EEF9002840F0C8808749204600F0E7F922
S1134E00002840F01981F8BD8449204600F004FAD6
S1134E100028C2D07C4B53F826508049204600F02D
S1134E201FFA95F82830002BB7D195F82900FEF722
S1134E3017FCE8603046FFF75FFDAB6900220421F0
S1134E4028469847A9E73046FFF724FDB8E7744998
S1134E50204600F0E1F9E0B140F203632B8695F8B7
S1134E602830012B11D03046FFF746FDAB691BB14A
S1134E70EA69032128469847636923F0C02323F491
S1134E80F81343F470236361A8E73046FFF702FD8B
S1134E90ECE76449204600F0BFF9E0B140F2046356
S1134EA02B8695F82830012B11D03046FFF724FDCE
S1134EB0AB691BB1EA69032128469847636923F06B
S1134EC0C02323F4F81343F47023636186E7304668
S1134ED0FFF7E0FCECE75449204600F09DF9E0B10F
S1134EE040F205632B8695F82830012B11D030460B
S1134EF0FFF702FDAB691BB1EA6903212846984715
S1134F00636923F0C02323F4F81343F4702363612B
S1134F1064E73046FFF7BEFCECE7444B63615DE7B2
S1134F204349204600F078F900283FF45EAF364B41
S1134F3053F826503046FFF763FD2B7DEBB96B68C1
S1134F4001336B60EB68013BEB60EB682BB9AB6939
S1134F501BB1EA69002128469847EB68002B7FF4CF
S1134F6044AF3046FFF796FCAB69002B3FF43DAFEE
S1134F70EA6902212846984737E76B6802336B6079
S1134F80EB68023BEB60E0E72A49204600F044F975
S1134F9000283FF431AF1C4B53F82650AB68002B6C
S1134FA03FF42AAF164B53F826703046FFF7D2FB76
S1134FB02B7DF3B92B6801332B60AB68013BAB60ED
S1134FC0AB68002B7FF418AF2B6A1BB16A6A01210E
S1134FD028469847AB68002B7FF40EAF00220D499A
S1134FE0384600F0BCF801220B49384600F0B7F807
S1134FF002E72B6802332B60AB68023BAB60DFE750
S1135000986B000014000300AC4E00201300020053
S1135010150003001700030016000300140002002B
S113502011000200100002001200020000C01FC0A4
S113503015000200170002001049204600F0ECF8A9
S113504000283FF4E0AE0E4B53F82640A368002B33
S11350507FF4D9AE94F82830012B0BD03046FFF7FB
S11350600DFB236A002B3FF4CEAE626A0221204678
S11350709847C8E63046FFF7CFFAF2E71600020079
S1135080AC4E0020064B0361064B43610023836151
S1135090036243624FF470328262C362704700BF9E
S11350A00400000F00C01FC010B40C4602B14C1C19
S11350B0022C0CD0836923F0100343EA04138361A8
S11350C0036923F0005303615DF8044B70470369DF
S11350D043F000530361F7E7826901F0FE0322F015
S11350E0020213438361836923F0010301F0010188
S11350F01943816170478369C1F3002223F080431F
S113510043EA82738361C9B201777047836923F0EC
S11351108043C1F3002243EA827323F00043C1F3C6
S1135120402243EAC2738361C9B20177704783693D
S1135130DB0F1B020B80C269D2B213430B80704792
S113514083695B0D03F400730B808269D20F43EA19
S113515002230B80C269D2B213430B80704710B490
S11351608BB2090C013906290ED8DFE801F0040DD1
S1135170100D0D1A2400016901249C4021EA040148
S113518002FA03F30B4303615DF8044B7047816932
S113519001249C4021EA040102FA03F30B438361D6
S11351A0F2E7416A01249C4021EA040102FA03F374
S11351B00B434362E8E7816A01249C4021F44031B7
S11351C021EA040102FA03F30B438362DCE70B0CCC
S11351D0013B062B1ED8DFE803F0041D0B1D1D1137
S11351E01700036988B223FA00F000F00100704749
S11351F0806989B2C84000F001007047406A89B2F2
S1135200C84000F001007047806A89B2C84000F0CD
S113521001007047002070470B0C023B052B1DD882
S1135220DFE803F0031C0A1C1016436988B223FA52
S113523000F000F001007047C06989B2C84000F076
S113524001007047406A89B2C84000F0010070470D
S1135250806A89B2C84000F001007047002070479E
S1135260474B994250D023D8033B994260D00FD882
S1135270023B994270D0013399427FD1436923F0B4
S1135280C02323F4F81343F4004343610020704720
S11352903C4B994242D0013399426FD1436923F088
S11352A0C02323F4F81343F48023436100207047A0
S11352B0354B994246D00FD80B3B99421AD00A334A
S11352C099425BD1436923F0C02323F4F81343F0DC
S11352D080434361002070472C4B994246D00133F0
S11352E099424BD1836A23F4403343F400338362FD
S11352F000207047436923F0C02323F4F81343F4D8
S11353008013436100207047436923F0C02323F4D2
S1135310F81343F40023436100207047436923F0EA
S1135320C02323F4F81343F400334361002070478F
S1135330436923F0C02323F4F81343F48033436117
S113534000207047436923F0C02323F4F81343F08B
S11353500043436100207047436923F0C02323F4D2
S1135360F81343F48043436100207047836A23F4B5
S1135370403343F480338362002070470120704738
S113538013000200110002001F00020010000700B9
S113539038B505460C460A460949FFF7E0FE2246A1
S11353A008492846FFF7DBFE224607492846FFF74F
S11353B0D6FE224605492846FFF7D1FE38BD00BF78
S11353C01B000300180003001A0003001900030067
S11353D008B50020FFF7D6FC08BD08B50120FFF78B
S11353E0D1FC08BD08B50220FFF7CCFC08BD60B1B4
S11353F070B506460C460025204600F043F80135FA
S11354001834AE42F8D1002070BD00207047C1604E
S113541070470000194B984204D0194B984220D091
S1135420FF207047102927D8DFE801F0090C262651
S11354302626262626262626260F1215180042F092
S11354400100704742F00200704742F004007047C8
S113545042F00800704702F00E00704702F00D00A1
S1135460704719B1012904D0FF20704702F00B00E6
S1135470704702F007007047FF20704700A0044007
S113548000B0044038B504460068616850F8212033
S1135490237A012B3FD0002B3AD0022B40D0657ADF
S11354A02D0105F0100322F050051D43A37A9B0142
S11354B003F040032B4323F4E065E37A082B32D056
S11354C01B0203F4E0632B43227BD20392B223F446
S11354D078231343627B120402F470221343A27BE9
S11354E00AB143F080732268616842F82130216870
S11354F0D1F8C02060680123834022EA0302E37BE1
S113550083401343C1F8C030E37A012B21D038BD66
S113551022F00202C3E722F0010242F00202BEE7D7
S113552042F00302BBE71B4B5A6802F00F02FFF77D
S113553071FFFF280BD0174B5A6822F00F025A60F4
S11355405A6800F00F00104358600023B8E70023A6
S1135550B6E721694B69227D22B1012A0AD0012ACA
S113556005D10BE0616801228A4023EA0203226923
S11355705361CCE760680122824013436568086880
S11355800122AA4020EA0200627DAA4002430A6086
S1135590EDE700BF00800440124BD3F8003623F03F
S11355A00103114A12780AB143F001030D4AC2F80B
S11355B00036D2F8003323F001030C4A12780AB102
S11355C043F00103074AC2F80033D2F8003123F054
S11355D00103074A12780AB143F00103014AC2F8F1
S11355E00031704700400640BB4E0020B94E0020F9
S11355F0BA4E0020094BD3F8002622F00102C3F86A
S11356000026D3F8002122F00102C3F80021D3F8C8
S1135610002322F00102C3F8002370470040064033
S11356200378042B13D000B583B004238DF8003025
S11356300123ADF802300223ADF80430ADF8063092
S113564069460020FDF7B2FC03B05DF804FB0020BE
S11356507047000010B582B000238DF805308DF836
S113566004301E4B1A79CAB11868031F013AD2B22A
S113567000EB8200012406E01278022A0BD0052AEE
S113568009D083420AD053F8042F11780029F3D1AA
S11356908DF80540F0E78DF80440F2E7104A93785E
S11356A003F0FE03937001A90E4800F075FA0E4B47
S11356B0D3F8002602F001020C490A70D3F8002343
S11356C002F001020A490A70D3F8003103F0010321
S11356D0084A1370002002B010BD00BFBC4E002069
S11356E000D0074000E0074000400640BB4E0020C9
S11356F0B94E0020BA4E0020074B5B69DBB2042B85
S113570006D0802B06D0012B0CBF01200620704749
S1135710022070470020704700E0074030B583B096
S11357200378022B16D90546B04A5269D2B2042A2C
S113573000F0C680102A00F00C81012A00F0678175
S1135740032B05D3042B40F20D81052B00F0C880F8
S113575004242DE1A54A5269D2B2042A00F0EF8054
S11357600DD8012A00F02B81022A40F05C8102222C
S1135770012B55D093B1022B6FD0042418E1102AC9
S113578000F04F81802A40F04E81012B3CD00BB9B0
S113579000240DE1022B5DD0042409E102A90123B8
S11357A001F8083D914800F079F90446002840F0DA
S11357B0FF8008E10124FBE0062B02D08C4B1B7810
S11357C003B38C4B1B78A3B1FFF7E6FE8A49002094
S11357D0FDF7ECFB0446002840F0EA800023854AEC
S11357E0137002A901F8043D804800F057F90446FB
S11357F0DEE002A9002301F8043D7C4800F04EF9E4
S11358000446D5E00124D3E0802300E00423012BE7
S113581006D1784B1B787BB90024C9E00123F6E755
S113582002A9012301F8083D704800F037F9044645
S1135830002840F0BD80ECE7FFF7AEFE6E49002083
S1135840FDF7B4FB0446002840F0B2800022694B07
S11358501A70ADE0802200E00422042A2ED0634BAB
S11358605B69DBB2012B0AD002A9012301F8083DD0
S11358705E4800F013F90446002840F099805D4B1F
S11358801B78BBB15C48FFF7CBFE0446002840F010
S11358908F800122574B1A7002AC022304F8083D92
S11358A0FFF7A8FE2146514800F0F8F804467FE0CF
S11358B00122D2E75048FDF7FBFBE3E7002477E041
S11358C0032B3AD3042B07D9052B36D1FFF714FF4A
S11358D0012813D000240DE004233FE001233DE020
S11358E002A9012301F8043D404800F0D7F804461A
S11358F00028EBD005238DF8043044E03D4B1B78A1
S113590073B13D48FFF78CFE04460028F2D1012212
S1135910384B1A7005238DF80430FFF76BFEE9E766
S11359203548FDF7C5FBECE74FF0E022D2F8103D17
S113593023F00203C2F8103D31E0042438E0012BC7
S11359403FF464AF002B3FF429AF022B84D004242E
S11359502EE0032B31D3042B2DD81023012B08BFA9
S1135960002407D002A9012301F8043D1F4800F0D8
S113597095F804462B788DF80430032B0CBF0123D3
S113598002238DF805309CB96B78002BCCD04FF0F6
S1135990E022D2F8103D43F00203C2F8103D01A901
S11359A0124800F07BF8041E40F2011318BF1C4695
S11359B0204603B030BD052B92D00424F8E7012B18
S11359C03FF42CAFF3B90D4BDB69C3F303630C4A0B
S11359D01278002A7FF4F0AE054A1278002A3FF4C8
S11359E0E9AE062B7FF4EAAE0124E1E700E00740CC
S11359F0B94E0020B84E0020CC4E00200040064096
S1135A00BB4E0020022B3FF453AF0424D0E7032BFA
S1135A1005D3042B7FF662AF052B3FF457AF042464
S1135A20C6E71022A4E6FF22A2E600BF2DE9F0415A
S1135A3080290BD05AB300244FF004084FF0FF0E16
S1135A404FF0100C8027012602250FE06423013B50
S1135A50FDD1EFE7102B16D0802B10D13B4600E090
S1135A602B46994214D00134A24211D04369DBB2CF
S1135A70042B06D0EED8012B07D0022BF0D07346AE
S1135A80EFE74346EDE76346EBE73346E9E70024F7
S1135A90A24294BF00200120BDE8F08108B50B7834
S1135AA0052B75D8DFE803F02F0317434343394A26
S1135AB0937803F0FE039370C36823F06003C3601C
S1135AC04FF47A720121FFF7B1FF002840F2011070
S1135AD018BF002008BD2F4A937803F0FE0343F05B
S1135AE001039370C36823F0600343F04003C36071
S1135AF04FF47A720421FFF799FF002840F2011055
S1135B0018BF002008BD234A937803F0FE03937066
S1135B10C36843F06003C3604FF47A728021FFF7D7
S1135B2085FF002840F2011018BF002008BD033B88
S1135B30DBB2012B22D9174A937803F0FE0343F01A
S1135B40010393700223C26822F007021343C36067
S1135B504FF0E022D2F8103D43F00403C2F8103DA8
S1135B6030BF4369DBB2012B0A4A937803F0FE038A
S1135B7018BF43F001039370002008BD026922F0AE
S1135B80C0024B789B01DBB2134303610023DAE7C5
S1135B90042008BD00D007400B78002B0CBF002365
S1135BA020234A780AB143F08003836070470000E1
S1135BB02DE9F04F83B08379012B07D0EBB1022B91
S1135BC015D001274FF0000B5E4604E0204B1E7BEE
S1135BD0022740F2031B00230B70002E2FD09146A6
S1135BE00C4680469A461A4DCDF804B011E0184B85
S1135BF01E7B01274FF4827BEDE7154B1E7B0227AA
S1135C0040F2031BE7E723780133DBB223709E42A3
S1135C1019D9AA6852F82330002BF4D01A79BA4261
S1135C20F1D01A689968404690470028EBD0237851
S1135C306B73B9F1010F05D1DDF804A0E3E74FF070
S1135C40000A00E0DA46504603B0BDE8F08F00BF1A
S1135C50BC4E002010B5094C206021710021A173B5
S1135C6032B11146A16023736373FFF7F3FC10BDD7
S1135C70024B00229A601A735A73F6E7BC4E002056
S1135C80F0B585B006460C4600238DF80F301B4B4B
S1135C901A6852F820701A7B5A738DF809108DF81F
S1135CA00800019701238DF80A300A460DF10F010F
S1135CB001A8FFF77DFF012C01D0054688B93846BD
S1135CC0FFF72CFD054660B90C4B9E7302238DF83B
S1135CD00A3001220DF10F0101A8FFF769FF054603
S1135CE008E000238DF80A3001220DF10F0101A80C
S1135CF0FFF75EFF284605B0F0BD00BFBC4E002094
S1135D00024A136801331360704700BFD44E002069
S1135D1070B582B004460D46002602A941F8046D10
S1135D203046FDF775FA144A16601449019BA1FB2D
S1135D3003139B0953609660072313601DB92378EE
S1135D407BB9032016E00E4B19681A46237843B931
S1135D501368B5F1FF3FF9D05B1A9D42F6D20320D8
S1135D6008E0FDF7FFFF2378013BDBB22370FDF76A
S1135D70EBFF002002B070BD10E000E0D34D6210D4
S1135D80D44E002010B50446FDF7ECFF2378DBB2B7
S1135D90FF2B08D023780133DBB223700024FDF7F6
S1135DA0D3FF204610BD0124F9E738B504460D465B
S1135DB0FDF7D8FF2570FDF7C7FF002038BD0000B0
S1135DC008B5FBF77DFBFBF761FA054A1368002B66
S1135DD0FCD0034A1368002BFCD0014B186808BDA3
S1135DE0F04E002010B5431E0A44914200D110BD6C
S1135DF011F8014B03F8014FF7E7024403469342BD
S1135E0000D1704703F8011BF9E710B59AB04FF4BD
S1135E100274019105916FF00041039106914FF6D0
S1135E20FF71ADF8121001A9ADF8104000F06CF844
S1135E30019B00221A701AB010BD000013460A46D6
S1135E40014602480068FFF7E0BF00BF6C07FF1F70
S1135E502DE9F0478E689E4282460C46914698464C
S1135E6035D88A8912F4906F31D0256809696F1A80
S1135E706569022305EB450595FBF3F508F101037C
S1135E803B449D4238BF1D46530531D5294600F099
S1135E902DFB064650B90C23CAF80030A38943F001
S1135EA04003A3814FF0FF30BDE8F0873A462169F3
S1135EB0FFF798FFA38923F4906343F08003A38141
S1135EC0266165613E44ED1B2660A5604646464555
S1135ED028BF464632464946206800F09FFAA36828
S1135EE09B1BA36023681E4426600020BDE8F08746
S1135EF02A4600F059FB06460028E1D121695046A4
S1135F0000F0A6FAC7E700002DE9F04F9DB08046E7
S1135F1003938B891C060D4616460FD50B696BB986
S1135F20402100F0E3FA2860286128B90C23C8F85E
S1135F3000304FF0FF30C5E040236B61002309932C
S1135F4020238DF8293030238DF82A304FF0010BAF
S1135F5037463C4614F8013B002B3CD1B7EB060A0C
S1135F600BD05346324629464046FFF771FF0130B5
S1135F7000F0A380099B534409933B78002B00F065
S1135F809C8000234FF0FF320493079305920693FD
S1135F908DF853301A93052221785048FAF7F0FB14
S1135FA0671C049BD8B9D90644BF20228DF853201E
S1135FB01A0744BF2B228DF8532022782A2A16D0A0
S1135FC0079A00210A20274601343B78303B092BED
S1135FD051D9C9B111E0252BC0D02746B9E73F4AB2
S1135FE0801A0BFA00F0184304903C46D3E7039A56
S1135FF0111D12680391002A01DB079204E052424A
S113600043F00203079204933B782E2B0ED17B7846
S11360102A2B07F1010132D1039B1A1D1B6803923D
S1136020002BB8BF4FF0FF33023705932C4C39785F
S113603003222046FAF7A4FB38B14023001B03FADD
S113604000F0049B034304930137397825488DF805
S1136050281006227E1CFAF793FB002835D0224B29
S1136060FBB9039B073323F0070308330393099B0E
S11360704B4409936CE700FB02320121A3E70023A0
S1136080059318460A240F4601313A78303A092A12
S113609003D9002BCAD00590C8E704FB00200123D4
S11360A0F1E703AB00932A46104B04A94046AFF333
S11360B00080B0F1FF3F8146D9D1AB895B063FF543
S11360C038AF09981DB0BDE8F08F03AB00932A46A2
S11360D0064B04A9404600F081F8EAE7AE6B0000E5
S11360E0B46B0000B86B000000000000515E0000BB
S11360F02DE9F04791461F468A680B69DDF8208038
S11361009342B8BF1346C9F8003091F843200646BD
S11361100C4612B10133C9F800302368990642BF16
S1136120D9F800300233C9F80030256815F00605A7
S113613007D104F1190AE368D9F800209B1A9D429B
S113614029DB94F843302268003318BF01239206F8
S11361502ED404F1430239463046C047013021D0E1
S11361602368E568D9F8002003F00603042B08BF70
S1136170AD1AA36822690CBF25EAE5750025934290
S1136180C4BF9B1AED184FF000091A344D451BD1BA
S11361900020BDE8F0870123524639463046C04707
S11361A0013003D14FF0FF30BDE8F0870135C2E77D
S11361B0E1185A1C302081F84300224494F8451019
S11361C082F843100233C4E701232246394630469D
S11361D0C0470130E6D009F10109D7E72DE9F043C2
S11361E017460A7E85B06E2A984606460C460C9BD6
S11361F001F1430C00F0BC801AD8632A2ED00AD8CF
S1136200002A00F0C880582A00F08A8004F1420570
S113621084F842202AE0642A01D0692AF6D1216850
S11362201A6811F0800F23D0111D1960136827E03C
S1136230732A00F0B48008D86F2A2AD0702AE5D1D6
S11362400A6842F020020A6003E0752A21D0782A05
S1136250DCD1782284F845206E4964E01A6801F1A3
S11362604205111D1960136884F842300123A3E02C
S113627011F0400F02F104011960D7D0B2F90030D7
S1136280002B03DA2D225B4284F8432062490A2260
S113629017E02068196810F0800F03D0081D1860FB
S11362A00B6806E010F0400F01F104001860F7D00D
S11362B00B8859496F2A14BF0A220822002084F847
S11362C043006568A560002DC0F29C80206820F022
S11362D004002060002B3FD1002D40F095806546DE
S11362E0082A0BD12368DA0708D5236962689A4221
S11362F0DEBF302305F8013C05F1FF35ACEB0503A7
S11363002361CDF800803B4603AA21463046FFF7BF
S1136310EFFE013055D14FF0FF3005B0BDE8F083FA
S113632081F845203C492268186812F0800F00F17A
S113633004051D6001D0036802E05506FBD50388FF
S1136340D00744BF42F0200222601BB9226822F029
S1136350200222601022B1E76546B3FBF2F002FB93
S11363601033CB5C05F8013D03460028F5D1B7E7AF
S113637008681A68496910F0800F04D0101D18606D
S11363801368196007E010F0400F02F10400186070
S11363901368F6D01980002323616546B1E71A68B3
S11363A0111D19601568626800212846FAF7E8F99A
S11363B008B1401B606063682361002384F84330A4
S11363C09FE723692A4639463046C0470130A2D0A8
S11363D023689B0707D5002504F11909E368039A8C
S11363E09B1A9D4205DBE068039B9842B8BF1846A0
S11363F093E701234A4639463046C04701308AD0E4
S11364000135EBE7002BA7D10B7884F8423004F177
S1136410420565E7D06B0000BF6B0000884210B5F1
S113642001EB020303D8421E99420CD110BD9842DD
S1136430F9D28118D21AD34200D110BD13F8014DFC
S113644001F8014DF7E711F8014B02F8014FEBE7B2
S113645038B50546002945D051F8043C0C1F002BE3
S1136460B8BFE41800F0D6F81F4A1368104633B9D1
S1136470636014602846BDE8384000F0CCB8A342FD
S11364800CD921686218934204BF1A685B68636080
S113649004BF521822600460ECE713465A680AB13C
S11364A0A242FAD919685818A0420BD120680144B5
S11364B0581882421960DDD1106852685A6001444C
S11364C01960D7E702D90C232B60D3E72068211881
S11364D08A4204BF11685268626004BF09182160CF
S11364E05C60C7E738BD00BF105F002070B5CD1CED
S11364F025F0030508350C2D38BF0C25002D064664
S113650001DBA94203D90C233360002070BD00F0E5
S113651081F8234A1468214691B9224C23681BB997
S1136520304600F067F820602946304600F062F8F3
S1136530431C26D10C233360304600F06CF8E4E7AA
S11365400B685B1B1AD40B2B0FD90B60CD50CC18E6
S1136550304600F060F804F10B00231D20F0070022
S1136560C31A1BD05A42E25070BD8C420DBF6368FF
S11365704B686360136018BF0C46E9E70C46496832
S1136580CAE7C41C24F00304A04205D0211A3046F3
S113659000F030F80130CDD02560D9E770BD00BFE0
S11365A0105F0020145F0020F8B5074614460E461D
S11365B021B91146BDE8F840FFF798BF22B9FFF7AB
S11365C047FF25462846F8BD00F026F884420FD937
S11365D021463846FFF78AFF05460028F2D03146A7
S11365E02246FFF7FFFB31463846FFF731FFE9E764
S11365F03546E7E738B5064C0023054608462360D0
S113660000F014F8431C02D1236803B12B6038BD99
S11366101C5F00207047704751F8040C0028A0F15B
S11366200400BCBF0B58C01870470000044B196825
S1136630024609B903491960186802441A60704790
S1136640185F0020205F0020A8140020C824002028
S1136650E83400200004FF1F0104FF1F0204FF1F91
S1136660200D0A0D0A202053746172747570203055
S11366703A203C3C205333324B31347820626F6FE4
S1136680746C6F61646572206261736520736F66F8
S113669074776172652073656375726564203E3E2C
S11366A02063757272656E742076657273696F6E9D
S11366B03A20323032312F30372F3034200D0A0D4A
S11366C00A000000202053797374656D20426173C1
S11366D06520486172647761726520696E666F3AFD
S11366E0200D0A002020534F53435F434C4B5F66F9
S11366F072657175656E6379203D20256420487A42
S1136700200D0A002020434F52455F434C4B5F66E7
S113671072657175656E6379203D20256420487A21
S1136720200D0A0020204255535F434C4B5F667294
S1136730657175656E637920203D20256420487A53
S1136740200D0A002020534C4F575F434C4B5F668B
S113675072657175656E6379203D20256420487AE1
S1136760200D0A00202052554E204D6F6465203DB7
S11367702025640D0A0D0A0020205374617274757B
S11367807020313A205333324B2055415254256402
S11367902042617564205261746520697320256408
S11367A0206269742F7300000D0A202053746172F3
S11367B074757020323A204A756D7020746F20749D
S11367C06865206170706C69636174696F6E2073B1
S11367D065676D656E7420746F2072756E6E696E78
S11367E0672E2E2E0D0A0000202052554E204D6F8C
S11367F06465203D2025640D0A0000000D0A202058
S11368005374617274757020313A205333324B20C3
S11368105541525425642042617564205261746567
S11368202069733A202564206269742F73200D0A4D
S11368300000000020205374617274757020323A95
S1136840205333324B204170706C69636174696FFB
S11368506E205570646174652046696E697368655D
S113686064202120323032312F30372F30340D0A5A
S11368700D0A0D0A00000000202053746172747523
S11368807020333A206170705F656E747279203DB8
S113689020252E3478203A2068617665206E6F209A
S11368A070726F6772616D20746F2072756E212033
S11368B00D0A000020205374617274757020343AFC
S11368C020706C65617365206C6F61642061707009
S11368D06C69636174696F6E2070726F6772616D49
S11368E020210D0A0D0A0000000000000000100025
S11368F00000001000000014FFFFFFFF0000000074
S1136900C804FF1FD804FF1FE804FF1FF804FF1F7B
S11369100805FF1F1805FF1F2805FF1F3805FF1F67
S1136920104D0020204D0020304D0020404D00200F
S1136930504D0020604D0020704D0020804D0020FF
S11369400000FF00FA0000000000000000C2010087
S1136950000000000203000000C20100000000006B
S11369600405000000C2010000000000060700004A
S11369700000000000000000000000000000000013
S11369800000000000000000000000000000000003
S113699000000000000000000000000000000000F3
S11369A000000000000000000000000000000000E3
S11369B000000000000000000000000000000000D3
S11369C00000730032002100610049004A004B00BE
S11369D04C004D003D000000240025002B00360033
S11369E03100000020000000380039003A00260081
S11369F06E006F0000003B0027005A00660037005D
S1136A002C002D002E0040006A006B006C0000007A
S1136A100000000000000000000000000000000072
S1136A2000FCAC06007E5603003FAB0100FCAC0644
S1136A30007E5603003FAB0100FCAC06007E56030B
S1136A40003FAB0100000000000000000000000057
S1136A5000000000000000000000000000FCAC0684
S1136A60007E5603003FAB01000000000000000060
S1136A700000000000B4C404006CDC02B0F3960112
S1136A8000B4C404006CDC02B0F3960100B4C40486
S1136A90006CDC02B0F3960100000000000000006E
S1136AA000000000000000000000000000000000E2
S1136AB000B4C404005A6202B0F39601000000005E
S1136AC0000000000000000000093D0000093D0036
S1136AD040420F0000093D0000093D0040420F0004
S1136AE000093D0000093D0040420F000000000085
S1136AF00000000000000000000000000000000092
S1136B000000000000093D0000093D0040420F0064
S1136B100000000000000000000000000000000071
S1136B200000000000000000000000000000000061
S1136B30004141414141000000202020202020202C
S1136B402020200040404040400080004848484801
S1136B50484800303030303030303036303030005B
S1136B600000000000000102030405060708090AEA
S1136B700B0C0D0E0F0000000000010002000300CA
S1136B800400050006000700080009000A000B00C5
S1136B900C000D000E000F0000A0064000B00640DF
S1136BA000C006404C4D4E001F0021002300232D41
S1136BB0302B2000686C4C00656667454647003002
S1136BC0313233343536373839414243444546004F
S1136BD0303132333435363738396162636465664F
S1136BE000000000F8B500BFF8B500BF00000000C9
S10B6BF05FF800F04D08FF1FDF
S10B6BF89498FF7F01000000E6
S1136C000101010001010101000100000101000076
S1136C100100010000127A000001000301010000DC
S1136C200001000000001800010100000100000044
S1136C30000000000100000003010301010603003D
S1136C40010203010106000101000000010000012E
S1136C50010000000100000000000000000000002E
S1136C600000000001010101010101010000000018
S1136C700E0000008004FF1F010100000404FF1F38
S1136C802B010000002C0100000047010100004816
S1136C900103000049010300004A010300004C0104
S1136CA00100004D010100004E010100002D010012
S1136CB000002E010000002F010000003001000040
S1136CC00031010000000000FF000000000000008F
S1136CD00000000000000000FF01030000000000AD
S1136CE00000000000000000FF020200000000009D
S1136CF00000000000000000FF030300000000008B
S1136D000000000000000000FF0404000000000078
S1136D100000000000000000FF0505000000000066
S1136D200000000000000000FF0606000000000054
S1136D300000000000000000FF0707000000000042
S1136D4000000000000000000001000064000000DA
S1136D50010000000000000000000000010000002D
S1136D6000010000F4010000010000000100000027
S1136D70000000000100000000010000E803000022
S1136D8001000000020000000000000001000000FB
S1136D9000010000A08601000100000003000000C3
S1136DA0000000000100000000C0044000000000DA
S1136DB00000000100000000C0F00F4001000000CE
S1136DC0009004401B0000000000000400000000CC
S1136DD00000000000000000009004401C000000BF
S1136DE0000000040000000000000000000000009B
S1136DF0009004401E00000000000001000000009C
S1136E0000F00F400101000000C004401000000029
S1136E100000000100000000C0F00F40010000006D
S1136E2000C004400F00000000000001000000004A
S1136E30C0F00F400100000000C004400E0000003C
S1136E40000000030000000000000000000000003B
S1136E5000C004400D00000000000003000000001A
S1136E600000000000000000009004400900000041
S1136E70000000020000000000000000000000000C
S1136E800090044008000000000000020000000020
S1136E9000000000000000009C06FF1F010000002D
S1136EA04301020000440102000029010000002AFD
S1136EB0010000002B010000002C0100000034013F
S1136EC00000003501000000360100000045010209
S1136ED000003A010000003C010200003D010200F4
S1136EE0003E010200003F010200004001020000D8
S1136EF0410102000046010200004701020000486F
S1136F000102000049010200004A010200004B0195
S1136F100200004C010200004D010200004E01027B
S1136F200000370100000038010000002D010000BE
S1136F30002E010000002F010000003001000000BD
S1136F4031010000003201000000000000C00240D6
S1136F5000D0024000E00240D1530000DB530000A7
S1136F60E553000000000200FFFFFF0F7007FF1F42
S1136F70000000000000000000000000000000000D
S1136F8000000000000000000000000000000000FD
S1136F9000000000000000000000000000000000ED
S1136FA000000000000000000000000000000000DD
S1136FB000000000000000000000000000000000CD
S1136FC000000000000000000000000000000000BD
S1136FD0054B5B7813F0800F04D1034A537843F0D8
S1136FE080035370704700BF000002400122034B2E
S1136FF0DA60034A1368013313607047007003407A
S11370009814002008B50821002000F03DF8024A39
S113701013680133136008BDA414002008B50421CB
S1137020002000F031F8024A13680133136008BDF0
S1137030A014002008B50221002000F025F8024A1F
S113704013680133136008BD9C14002038B505464D
S11370500B4A137843F0800313701446237813F01B
S1137060800F05D1AB69B3F1FF3FF7D09847F5E73F
S1137070034B1B7813F0710F14BF0120002038BD9F
S113708000000240000000005FF800F0C140000072
S9030411E7
